:020000040000FA
:1000000085EF07F01200FFFF04EF10F01200FFFF72
:10001000FFFFFFFFFFFFFFFF0CEF10F01200FFFFDD
:10002000FFFFFFFFFFFFFFFFFFFF00000401105174
:10003000600BE842E842E842E842E842000901E099
:1000400055D01151070A51E00B0A4FE0070A40E072
:10005000010A2CE00B0A28E0020A26E0030A22E04B
:10006000080A12E0010A0EE00F0A0AE0030A01E0A2
:100070003CD00001010EB06F0001040EB76F36D006
:1000800036D834D090D832D00001010EB06F0001C4
:10009000B90EB16F000EB26F0001B8930001010EEE
:1000A000B56F24D0A8D822D0F5D820D00001010EF9
:1000B000B06F040114510001B16FB26BBA0EB127D9
:1000C000000EB2230001B8930001010EB56F0ED0EF
:1000D0000001010EB06F04011451EA6ABA0FE96E13
:1000E000000EEA2212C4EFFF01D000D01200800EF1
:1000F0000401105D57E11351030A34E0010A10E0D6
:10010000030A01E04DD00001010EB06F0001600E46
:10011000B16F0C0EB26F120E0001B56FB66B40D00E
:100120000001010EB06F04011251F66EF76AD8900B
:10013000F636F7369E0EF6260D0EF7220900F5CF9D
:10014000B1F00A00F5CFB2F0020E0001F76AB12556
:10015000F66EB251F7220900F5CFB5F00A00F5CFDF
:10016000B6F01ED00001010EB06F04011251F66E00
:10017000F76AD890F636F736A20EF6260D0EF7225D
:100180000900F5CFB1F00A00F5CFB2F0B1C0F6FF2B
:10019000B2C0F7FF0800F5500001B56FB66B00D094
:1001A0000001B88312000001010EB06F0F0EE66E61
:1001B000710EE66E0F0EE66E1BEC06F0E552E55290
:1001C000E552010EE66EBA0EE66E000EE66E1BEC10
:1001D00006F0E552E552E55212C4B9F0040112519D
:1001E00004E10001050EB76F05D00001060EB76FE0
:1001F000E7EC04F012000401186B196B04011051B4
:100200001F0B020A15E0030A0FE0010A01E034D0D7
:100210000001010EB06F02D0040118810001B8A1E5
:1002200002D00401188328D00001010EB06F24D041
:100230000001010EB06F040114510F0B080DF350B3
:10024000016A000F006E040E01221451800B01E0C0
:10025000010E040DF35000010024B36F000E0120C5
:10026000B46FB3C0E9FFB4C0EAFFEF50040B03E082
:100270000401010E186F00D00001B0050AE1000171
:10028000180EB16F040EB26F0001B8930001020E98
:10029000B56F12000401120510E110511F0B000987
:1002A0000CE10001010EB06F030E0401115D03E1CA
:1002B0000001B88102D00001B891040112513AE165
:1002C00010511F0B020836E114510F0B000932E0E8
:1002D0000001010EB06F040114510F0B080DF35013
:1002E000016A000F006E040E01221451800B01E020
:1002F000010E040DF35000010024B36F000E012025
:10030000B46F030E0401115D07E1840EB3C0E9FF71
:10031000B4C0EAFFEF6E0ED014AF06D0B3C0E9FF51
:10032000B4C0EAFFEF6A06D0880EB3C0E9FFB4C0DC
:10033000EAFFEF6E12006C500BE1040100513C0B20
:10034000E842E8420D0802E108D801D03CD804D0C8
:10035000040E6C5C01E147D81200D9CFE6FFE1CF73
:10036000D9FFE6520001AF6BB06BB56BB66B16EC04
:1003700000F0DF6ADF50006E016A010E005C000EC3
:1003800001581BE20001B05101E017D0F76ADF34D9
:10039000FE0BF736F66EAC0EF6260D0EF7220900B0
:1003A000F5CF00F00800F5CF01F004D001C0FAFF4E
:1003B0000050F96EFBDFDF2ADDD7D5D8E552E552D4
:1003C000E7CFD9FF1200020E0001AF5D0AE192D81B
:1003D000040100BD03D0C80E006F02D0880E006F6C
:1003E00001D007D91200040E0001B75D0AE112C462
:1003F0006EFF6E50000803E2050EB76F02D0030EC9
:10040000B76F0001AF050AE10BD8040104BD03D0AA
:10041000C80E046F02D0880E046F01D0EAD8120013
:10042000D9CFE6FFE1CFD9FF020EE1260001080E89
:10043000B55D000EB65905E2B5C0DEFFB6C0DDFF02
:1004400003D0080EDE6EDD6A040104930491010EF0
:10045000DB500413DFCF05F4000EDB500001B55F65
:10046000010EDB50B65B180EB36F040EB46F0001C3
:10047000B8A31ED0D9CFE9FFDACFEAFFEE50ED10D6
:1004800016E0B1C0F6FFB2C0F7FF0800F550B3C0E8
:10049000E9FFB4C0EAFFEF6E0001B32B000EB423F6
:1004A000B12BB223DF06010E01E2DB06E3D71CD03D
:1004B000D9CFE9FFDACFEAFFEE50ED1015E0B1C079
:1004C000E9FFB2C0EAFFEF50B3C0E9FFB4C0EAFFF2
:1004D000EF6E0001B32B000EB423B12BB223DF0665
:1004E000010E01E2DB06E4D7D9CFE1FFE552E7CF09
:1004F000D9FF1200D9CFE6FFE1CFD9FF020EE126E6
:10050000030E04010015E76E010EE7CFDBFF01C407
:10051000DFFFDE500001B527DD50B623180EB16FA6
:10052000040EB26FD9CFE9FFDACFEAFFEE50ED103B
:1005300014E0B1C0E9FFB2C0EAFFEF50B3C0E9FF79
:10054000B4C0EAFFEF6EB32B000EB423B12BB2237D
:10055000DF06010E01E2DB06E5D7D9CFE1FFE55268
:10056000E7CFD9FF12006D980001B0510CE10401F2
:10057000080E016F100E026F040E036F840E006FE1
:100580000401046F35D0040110AF22D00001B55131
:100590000401165D0001B6510401175904E216C4A6
:1005A000B5F017C4B6F03CDF0001010EAF6F0401D7
:1005B000080E016F100E026F040E036F800E006FA5
:1005C0000401180E066F040E076FC80E046F10D0DA
:1005D0000001020EAF6F0401056BC80E046F040129
:1005E000080E016F180E026F040E036FC80E006F25
:1005F00012000001AF6B0401080E016F100E026FB4
:10060000040E036F880E006F0401046B1200550E78
:10061000A76EAA0EA76EA68212000001420E6A6F94
:10062000020E6B6F010E6C6F12000001606B665161
:10063000605D1EE260C000F0016A026A675100243A
:10064000F36E68510120F46E69510220F86EF4CF08
:10065000F7FFF3CFF6FF0800F5CF61F06051EA6ACB
:100660006A0FE96E000EEA2261C0EFFF602BDFD750
:10067000F86A1200840EA66E0001606B6651605D20
:1006800027E26051EA6A6A0FE96E000EEA22EFCFB4
:1006900003F060C000F0016A026A67510024F36E43
:1006A00068510120F46E69510220F86EF4CFF7FF13
:1006B000F3CFF6FF03C0F5FF0C001F0E60151F08F7
:1006C00003E06605605D01E1A2DF0001602BD6D783
:1006D00012000001606B6651605D20E2940EA66E10
:1006E0006051006E016A060ED89000360136E804AB
:1006F000FBE1026A01BE0268000167510024F36E4B
:1007000068510120F46E69510220F86EF4CFF7FFB2
:10071000F3CFF6FF7CDF0001602BDDD7F86A120013
:10072000A66A0001606B6651605D0EE2675160254C
:10073000A96EA6806051EA6A6A0FE96E000EEA228D
:10074000A8CFEFFF602BEFD712000001606B66515E
:10075000605D13E267516025A96E6051EA6A6A0F15
:10076000E96E000EEA22EF50A86E040EA66E4FDF6F
:10077000A6B2FED70001602BEAD71200C40EA66E07
:100780000001606B6651605D20E26051EA6A6A0FA9
:10079000E96E000EEA22EFCF03F060C000F0016ABC
:1007A000026A67510024F36E68510120F46E6951AA
:1007B0000220F86EF4CFF7FFF3CFF6FF03C0F5FF8A
:1007C0000C0025DF0001602BDDD7F86A1200400E17
:1007D000E66E650EE66E000EE66E36EC05F0E5524E
:1007E000E552E552000870E20001606B00016551BE
:1007F000FF0A57E0FA0A50E0010A3BE0070A34E03A
:10080000010A2DE0030A18E0070A16E0700A01E069
:100810005AD003DF0001040E606F04010CBFFDD746
:10082000400EE66E650EE66E000EE66EFCEC04F021
:10083000E552E552E55248D0F8DE050E000160278A
:1008400004010CBFFDD7400EE66E650EE66E000E8D
:10085000E66EFCEC04F0E552E552E55235D00ADFD5
:100860000001010E606F30D034DF0001010E606FB7
:100870002BD056DF050E0001602704010CBFFDD709
:10088000400EE66E650EE66E000EE66EFCEC04F0C1
:10089000E552E552E55218D058DF0001010E606FB5
:1008A00013D093EC05F00001636B646B00016307E8
:1008B000000E645B00016351641103E0000000005E
:1008C000F5D7FF0001D000D01200040110511F0B1A
:1008D000010801E079D0145101E076D0060E115DD7
:1008E0002EE11351230A28E0010A13E0030A01E074
:1008F00024D00001020EB06F0001B90505E100012E
:10090000840EB16F0C0EB26F090E0001B56FB66B9D
:1009100014D00001020EB06F0001B90505E100011D
:10092000810EB16F0D0EB26F0001B90504E11D0E0D
:100930000001B56FB66B01D000D00001B88304018F
:100940001051600BE842E842E842E842E842010800
:1009500001E03AD011510B0A31E0080A21E0090AFE
:1009600019E0080A09E00B0A05E0080A01E02CD0AA
:100970002CD82AD02BD828D00001020EB06F00014D
:10098000BB0EB16F000EB26F0001B8930001010EF3
:10099000B56F1AD00001020EB06F13C4BBF014D0B3
:1009A0000001020EB06F0001BC0EB16F000EB26FFD
:1009B0000001B8930001010EB56F06D00001020ED0
:1009C000B06F12C4BCF000D012001200120000017F
:1009D000BD6B1E0E716E0401400E096F200E0A6F72
:1009E000040E0B6F880E086F0401600E0E6F040E6C
:1009F0000F6F400E0C6F1200D9CFE6FFE1CFD9FF89
:100A0000E652FC0EDB50400805E2400EF36EFC0E91
:100A1000F3CFDBFFDF6AFC0EDB50DF5C19E2DF5057
:100A2000E76EFD0EDBCFE9FFFE0EDBCFEAFFE750FE
:100A3000E926000EEA22EF50E66EDF50EA6A600F08
:100A4000E96E040EEA22E552E750EF6EDF2AE3D7A3
:100A5000FC0EDBCF0DF4400E04010C170C7D880E4C
:100A60000C13E552E552E7CFD9FF1200D9CFE6FFCC
:100A7000E1CFD9FF0001BD6B040108BF30D0FC0EEF
:100A8000DBCF00F00951D880005403E2FC0E09C40A
:100A9000DBFF0001BD6BFC0EDB50BD5D19E2BD51FB
:100AA000EA6A200FE96E040EEA22EF50E66EBD51AD
:100AB000E76EFD0EDBCFE9FFFE0EDBCFEAFFE7506E
:100AC000E926000EEA22E552E750EF6EBD2BE3D790
:100AD0000401400E096F0817087D880E08130001F5
:100AE000BD5100D0E552E7CFD9FF12006DA60FD857
:100AF00002D06DB613D80001B70508E16DBA06D073
:100B0000686A696A69806988020EB76F12006D6A47
:100B1000696A6D860001010EB76F12006D6A696A1D
:100B20000001B76B12008EEF05F00001B75101E133
:100B30003AD06850040B04E06950040B01E038D847
:100B40006DB231D06850010B04E06950010B01E037
:100B500050D86850100B04E06950100B01E024D805
:100B60006850400B04E06950400B01E037D86850F2
:100B7000200B04E06950200B01E032D86850020BD2
:100B800004E06950020B01E032D8030E0001B75DAA
:100B900001E209D06850080B06E06950080B03E039
:100BA0009BEC01F068961200698468986D821200CF
:100BB0006D926994689412000001B8A10ED0F8DF1C
:100BC0006D840001080EBE6F070EBF6FBE07000EDA
:100BD000BF5BBE51BF11FAE16D941200689C120018
:100BE00070A003D0F9EC02F07090689A120068923D
:100BF00012006A6A686A9F0E6B6E7B0E696E6E6A7F
:100C00000F0EE66E710EE66E0F0EE66E14D8E5520C
:100C1000E552E552160E706E68A602D06896FCD7B3
:100C20006D98F9EC02F00001B8910001B96B000178
:100C3000030EB76F1200D9CFE6FFE1CFD9FFFD0E4B
:100C4000DBCFE9FFFE0EDBCFEAFFFC0EDB5004E05A
:100C5000EE6AFC0EDB06F9D7E552E7CFD9FF1200AA
:100C60001201000200000008D80433000100010254
:100C70000302090229000101028032090400000276
:100C800003000000092101000001221D0007058169
:100C90000340000107050103400001090220000193
:100CA000020480320904000002FF000000070581F1
:100CB0000340000107050103400001040309043457
:100CC000034D006900630072006F006300680069F3
:100CD000007000200054006500630068006E006F23
:100CE000006C006F0067007900200049006E00630F
:100CF000002E0048035000490043006B0069007457
:100D0000002000320020004D006900630072006F77
:100D10000063006F006E00740072006F006C006C66
:100D200000650072002000500072006F00670072C2
:100D30000061006D006D00650072001603500049EF
:100D400000430031003800460032003500350030E5
:100D50000030035000490043006B0069007400201C
:100D6000003200200043006F006E006600670075CF
:100D70000072006100740069006F006E0020003294
:100D8000000600FF0901A10119012940150026FFF5
:100D900000750895408102190129409102C0720C2A
:100DA0009B0CBB0CBF0CF30C3B0D510DCA082A0E5B
:100DB000F66E000EF76E000EF86E00010900F55099
:100DC000AA6F0900F550AB6F03E1AA6701D03DD0CF
:100DD0000900F550A56F0900F550A66F0900F55000
:100DE000A76F09000900F550E96E0900F550EA6E99
:100DF000090009000900F550A86F0900F550A96F16
:100E000009000900F6CFACF0F7CFADF0F8CFAEF0A7
:100E1000A5C0F6FFA6C0F7FFA7C0F8FF0001A853C2
:100E200002E1A95307E00900F550EE6EA807F8E2C9
:100E3000A907F9D7ACC0F6FFADC0F7FFAEC0F8FF09
:100E40000001AA07000EAB5BBFD71200D9CFE6FFA7
:100E5000E1CFD9FF030EE126938A818AF19E580ED5
:100E6000E66E6EEC07F0E55281AA0DD0FE0EF66E2E
:100E70007F0EF76EF86A0800F550DF6E550EDF5CE6
:100E800002E100EF10F018D822D8E7EC03F0D950B7
:100E9000010FE96EDACFEAFFEE50ED1001E18B7041
:100EA000010EDB06020E01E2DB06EED7D9CFE1FF31
:100EB000E552E7CFD9FF1200140E6F6E0001B76B39
:100EC0000001B86B0001B96B8B909490120076EC26
:100ED00005F06FBE02D095EC05F01200FF0EE35056
:100EE000076EEF0E01D0F30EE76EE72E75EF07F0F9
:100EF0000C0E066EE76AE72E7BEF07F0062E7AEF00
:100F000007F0072E73EF07F0120013EE00F023EE48
:100F100000F0F86A059CD7EC06F026EC07F0FDD748
:100F20001200FFFFFFFFFFFFFFFFFFFFFFFFFFFFBD
:100F3000FFFFFFFFFFFFFFFFFFFFFFFFFFFFFFFFC1
:100F4000FFFFFFFFFFFFFFFFFFFFFFFFFFFFFFFFB1
:100F5000FFFFFFFFFFFFFFFFFFFFFFFFFFFFFFFFA1
:100F6000FFFFFFFFFFFFFFFFFFFFFFFFFFFFFFFF91
:1020000072EF3EF0120000007BEF3AF01200000089
:1020100000000000000000007BEF3AF0120000001A
:10202000FFFFFFFFFFFFFFFFFFFFD9CFE6FFE1CF7D
:10203000D9FFE652030ED26EA194A08492809282C0
:102040000D0EC16E030EC06E9284809489949286A8
:102050008096899692888998899A929A8A96939678
:102060008A889398938A818AF19E8A9493948B901C
:1020700094908B9294928B949494949C8B8C1E6AE3
:102080000001E76B0001010EE86F0201030EE06F33
:102090000201E16B0201010EE26F8FEC19F071ECAD
:1020A00017F069EC17F043EC17F00001400ED880F0
:1020B000E355010EE4550EE30001C00EE35D000E92
:1020C000E45908E30001E651AF0804E3500E0001B3
:1020D000E65D09E20001E36B010EE46F0001E56BD0
:1020E0000001800EE66F080ED56E040ECA6E4F0E0C
:1020F000CB6E0C0EBD6E1D0EBE6E0001400EE06F6D
:1021000000013E0EE16F00013C0EE26F02017E0E07
:10211000FA6F02012D0EFB6F070EB46EB56AF28CDA
:10212000F28E71EC3BF0040EE66E3DEC2AF0E552C7
:10213000500825E1050EE66E3DEC2AF0E5524B080D
:102140001EE1060EE66E3DEC2AF0E552320817E17C
:10215000070EE66E3DEC2AF0E5521D6E020E1E6E75
:10216000546AE66A110EE66EB7EC15F0E552E552D8
:10217000400EE66EDCEC16F0E5520201FA6FE55215
:10218000E552E7CFD9FF120004010CBFFDD7400E86
:10219000E66E400EE66E020EE66EF6EC39F0E552A3
:1021A000E552E5526FEC3DF01200D9CFE6FFE1CFEA
:1021B000D9FF020EE126DF6A010EDB6A81BA02D086
:1021C0000001E78D400EE66E000EE66E020EE66E32
:1021D00032EC3AF0E552E552E552000803E2DE52F5
:1021E000010EDD6E1E0406E1010EDB5002E065EC1F
:1021F0002FF008D2020E1E5C09E1010EDB5004E054
:10220000760E0201005D02E007DAFCD10001E8B3BE
:102210007DDA010EDB5001E1F5D1DF50EA6A000FF3
:10222000E96E020EEA22EF50546E5450420A25E045
:10223000340A05E02C0A01E023D0DF2ADFD1020EA8
:102240001E5C17E18A881E6AE668040EE66E1BECC7
:102250002AF0E552E552E668050EE66E1BEC2AF020
:10226000E552E552E668060EE66E1BEC2AF0E552F2
:10227000E552E7EC1CF0DF2AC1D1AFEC1CF0BED177
:10228000A00E545C03E2400EDF6EB8D15450B90882
:1022900003E2400EDF6EB2D1A00E545E549E54464F
:1022A000F9505450F9261AD03FD06BD06ED071D06F
:1022B0007AD091D0B1D0B4D0BDD0C0D0C3D0C6D028
:1022C000C9D0CBD0CDD0D0D005D10DD115D11DD115
:1022D0001FD127D128D12FD17AD190D1DF28EA6A16
:1022E000000FE96E020EEA22EF50E66E020EDF24C6
:1022F000EA6A000FE96E020EEA22EF50E66EB7ECD2
:1023000015F0E552E552030EDF24EA6A000FE96E8C
:10231000020EEA22EF50E66EDCEC16F0E552020106
:10232000FA6F040EDF26D9D7DF28EA6A000FE96EBC
:10233000020EEA22EFCFE0F0020EDF24EA6A000F7D
:10234000E96E020EEA22EF50E66EDCEC16F0E55282
:10235000010F0001E16F020E0001E15D0001E26F7B
:10236000030EDF24EA6A000FE96E020EEA22EF5044
:10237000E66EDCEC16F0E5520201FB6F040EDF2680
:10238000ACD7C7EC1CF0DF2AA8D724EC18F0DF2A62
:10239000A4D7DF2AD9CFE6FFDACFE6FF29EC1AF07F
:1023A000E552E5529AD7DF2ADF28EA6A000FE96E84
:1023B000020EEA22EF50E66EDF50EA6A000FE96E85
:1023C000020EEA22EF50E66E3EEC19F0E552E552BD
:1023D000020EDF2682D7DF2ADF50EA6A000FE96E9D
:1023E000020EEA22EF50E66EDF28206A000F1F6E11
:1023F000020E20221FC0E6FF20C0E6FFF3EC1CF017
:10240000E552E552E552DF50EA6A000FE96E020E2E
:10241000EA22EF28DF2661D771EC17F0DF2A5DD7BB
:10242000DF2AD9CFE6FFDACFE6FFAAEC19F0E552B2
:10243000E55253D769EC17F0DF2A4FD79DEC18F01F
:10244000DF2A4BD78FEC19F0DF2A47D7F0EC18F0D2
:10245000DF2A43D7400EDF6E40D7FF00DF2A3DD78B
:1024600079EC17F0DF2A39D7DF28EA6A000FE96E26
:10247000020EEA22EF500001E36FE46B020EDF244C
:10248000EA6A000FE96E020EEA22EFCF1FF0206A1F
:102490001FBE20681FC020F01F6A1F500001E327E5
:1024A00020500001E423030EDF24EA6A000FE96EE6
:1024B000020EEA22EFCFE5F0040EDF24EA6A000FF5
:1024C000E96E020EEA22EFCFE6F020EC17F0050EDF
:1024D000DF2603D7DF2AD9CFE6FFDACFE6FFC5DA5A
:1024E000E552E552FAD6DF2AD9CFE6FFDACFE6FF8A
:1024F0003CDAE552E552F1D6DF2AD9CFE6FFDACF52
:10250000E6FF96D9E552E552E8D6DF2ADDD9E5D6D1
:10251000DF2ADFCFE6FF0FEC2FF0E552030EDF26B8
:10252000DCD6DF2ADAD6DF2ADFCFE6FF38D9E5525C
:10253000400EDF6ED2D6DF2ADF50DF2AEA6A000FB4
:10254000E96E020EEA22EF505F6EDF50DF2AEA6A80
:10255000000FE96E020EEA22EF50546EDF50DF2AC0
:10256000EA6A000FE96E020EEA22EF50566EDF5063
:10257000DF2AEA6A000FE96E020EEA22EF50586E77
:10258000DF50DF2AEA6A000FE96E020EEA22EF50FE
:10259000596EDF50DF2AEA6A000FE96E020EEA2266
:1025A000EF505A6EDF50DF2AEA6A000FE96E020E22
:1025B000EA22EF285B6EDF50DF2AEA6A000FE96E3D
:1025C000020EEA22EF505E6EB7EC2DF086D6DF2ABF
:1025D000DF28EA6A000FE96E020EEA22EF50E66E8B
:1025E000DF50EA6A000FE96E020EEA22EF50E66E53
:1025F0007BD9E552E552020EDF266FD6400EDF5C36
:1026000001E20BD6020EE15C02E2E16AE552E16E04
:10261000E552E7CFD9FF1200F29A870ED56EF2A4E9
:1026200029D0D20ED76E3A0ED66EF294542A545058
:10263000050801E2546A040E545C06E2010E5414CB
:10264000E8B08A88E8A08A98300E0001E71512E009
:102650008A8881BAFED78F0E0001E717F00EE66E6A
:1026600047EC3EF0E55281AAFED7F00EE66E47EC4D
:102670003EF0E5520001E7AD47D08A880DEC31F01D
:102680008A888A8681AAFED7546AE66A110EE66EA7
:102690006EDAE552E552400EE66E8EDBE55202013F
:1026A000FA6F300E0001E71502E081BAFED7FC0E8A
:1026B0000001E81506E0080EE66E4DEC36F0E55236
:1026C00010D0190406E1040EE66E4DEC36F0E5522A
:1026D00008D01650171005E0060EE66E4DEC36F0E9
:1026E000E552F00EE66E47EC3EF0E55281AAFED7C9
:1026F000F00EE66E47EC3EF0E5528F0E0001E71754
:102700000001E86B0001E79D8B901200D9CFE6FF36
:10271000E1CFD9FFE6521D501AE01D50DF6E1D6A51
:102720001A50E66EB6EC27F0E552DF50010805E2DC
:102730001B50E66EB6EC27F0E552DF50020805E2CA
:102740001C50E66EB6EC27F0E5521D50E6E10201A2
:10275000E551E61108E0A050020B05E1EBEC27F093
:10276000196EA182A0828150100B14E1C250020B9D
:1027700011E10201FA51C45C0AE20C0E0201FC5D97
:1027800003E18A948A8802D00201FC2B02D0020164
:10279000FC6BC282E552E552E7CFD9FF1200D9CFD8
:1027A000E6FFE1CFD9FFFE0EDBCFE6FF23EC2FF0F3
:1027B000E552000939E0020E1E6E546AE66A110EF7
:1027C000E66ED5D9E552E552400EE66EF5DAE552F1
:1027D0000201FA6F500EE66E040EE66E1BEC2AF054
:1027E000E552E5524B0EE66E050EE66E1BEC2AF046
:1027F000E552E552320EE66E060EE66E1BEC2AF04E
:10280000E552E552FE0EDB50030FEA6A000FE96E57
:10281000020EEA22EF501D6E1D50E66E070EE66EA8
:102820001BEC2AF0E552E552E552E7CFD9FF120042
:10283000D9CFE6FFE1CFD9FFF29E86EC3BF0050E43
:10284000C26EC282FD0EDBCFE9FFFE0EDBCFEAFFD8
:10285000EF50EF2AEA6A000FE96E020EEA22EF500B
:10286000146EFD0EDBCFE9FFFE0EDBCFEAFFEF506B
:10287000EF2AEA6A000FE96E020EEA22EF50156EA7
:10288000166A176A186A196A1A6A1D6A0001E883CB
:1028900092968986928492888A94899A2E0EB46E32
:1028A000A50EB56E0C0EE66E8EEC3EF0E5529D90D8
:1028B000A092910ECD6E910EB16EA19CA08CF28E65
:1028C000E552E7CFD9FF1200F29E0001E893A09CE9
:1028D0009D90A092CD6AB16A070EB46EB56A9286D9
:1028E00071EC3BF0F28E1200D9CFE6FFE1CFD9FFB9
:1028F000030EE126FD0EDB50216E226A21C022F07C
:10290000216AFE0EDB50000121241F6E000E2220E2
:10291000206E010E1FC0DBFF020E20C0DBFFDF6A4E
:10292000DF501F6E206AD890205004E6800E1F5C96
:10293000000E205810E2010EDBCFE9FFDB2A020E69
:10294000DBCFEAFF01E3DB2AEF50E66EB6EC27F0BF
:10295000E552DF2AE5D7030EE15C02E2E16AE552C7
:10296000E16EE552E7CFD9FF1200D9CFE6FFE1CF04
:10297000D9FF050EE126FD0EDBCFE9FFFE0EDBCF12
:10298000EAFFEF50EF2AEA6A000FE96E020EEA2230
:10299000040EEFCFDBFFFD0EDBCFE9FFFE0EDBCF3A
:1029A000EAFFEF50EF2AEA6A000FE96E020EEA2210
:1029B000EF50E66ED950020FE96EDACFEAFFE5522A
:1029C000E750EE6EED6AD950020FE96EDACFEAFFFA
:1029D000200ED880EE54000EED5407E2200EF36E68
:1029E000020EF3CFDBFF030EDB6AD950020FE96E54
:1029F000DACFEAFFEE50ED1001E12DD0DE6ADD6A9C
:102A0000DECF1FF0DDCF20F0020EDBCF21F0030E72
:102A1000DBCF22F021501F5C225020581AE2040E16
:102A2000DBCFF3FFDB2AF350E66E3DEC2AF0E552F4
:102A3000E66EDECFE9FFDDCFEAFF400EE926020EAB
:102A4000EA22E552E750EF6EDF2A010E01E3DB2AAE
:102A5000D7D7C4EC10F0050EE15C02E2E16AE55262
:102A6000E16EE552E7CFD9FF1200D9CFE6FFE1CF03
:102A7000D9FF050EE126FD0EDBCFE9FFFE0EDBCF11
:102A8000EAFFEF50EF2AEA6A000FE96E020EEA222F
:102A9000040EEFCFDBFFFD0EDBCFE9FFFE0EDBCF39
:102AA000EAFFEF50EF2AEA6A000FE96E020EEA220F
:102AB000EF50E66ED950020FE96EDACFEAFFE55229
:102AC000E750EE6EED6AD950020FE96EDACFEAFFF9
:102AD000200ED880EE54000EED5407E2200EF36E67
:102AE000020EF3CFDBFF030EDB6AD950020FE96E53
:102AF000DACFEAFFEE50ED1001E12FD0DE6ADD6A99
:102B0000DECF1FF0DDCF20F0020EDBCF21F0030E71
:102B1000DBCF22F021501F5C225020581EE2FD0E18
:102B2000DBCFE9FFFE0EDBCFEAFFEF50EF2AEA6AC8
:102B3000000FE96E020EEA22EF50E66E040EDBCFC4
:102B4000F3FFDB2AF350E66E1BEC2AF0E552E55268
:102B5000DF2A010E01E3DB2AD3D7050EE15C02E296
:102B6000E16AE552E16EE552E7CFD9FF1200D9CF15
:102B7000E6FFE1CFD9FF030EE126FE0EDB50226E09
:102B8000236A22C023F0226AFD0EDB5000012224BA
:102B90001F6E000E2320206E216A20BE21681FC0F8
:102BA000DFFF010E20C0DBFF020E21C0DBFFD9CF0B
:102BB000E9FFDACFEAFF060EE76ED890020EEB329D
:102BC000010EEB32EF32E706F8E1E5C01FF0206AB4
:102BD000216A1FAE02D020682168D9CFE9FFDACF81
:102BE000EAFF1F50EE262050EE222150EE22E6C0D2
:102BF0001FF0206A216AD9CFE9FFDACFEAFF1FC0B0
:102C00000CF020C00DF021C00EF0EECF07F0EECF9B
:102C100008F0EFCF09F016EC3DF006C0EDFF05C05F
:102C2000EDFF04C0EFFFD9CFE9FFDACFEAFFD8907C
:102C3000020EEB32010EEB32EF32080E226ED9CFCC
:102C4000E9FFDACFEAFF22501F0BEECF1FF0EECFE5
:102C500020F0EECF21F006E0D890213220321F3252
:102C6000E806FAE11F50BE6ED9CFE9FFDACFEAFFDE
:102C7000EE52EE6AEE6ACF0EBD14226E236A246A0B
:102C8000020E286ED9CFE9FFDACFEAFF28501F0BDA
:102C9000EECF25F0EECF26F0EECF27F006E0D8906D
:102CA000273226322532E806FAE1225025101F6E1F
:102CB00023502610206E24502710216E1F50BD6E09
:102CC000030EE15C02E2E16AE552E16EE552E7CF14
:102CD000D9FF1200D9CFE6FFE1CFD9FF040EE126DC
:102CE000FD0EDBCF1FF0FE0EDBCF20F0000E1FC06D
:102CF000DBFF010E20C0DBFF020EDB6A030EDB6A86
:102D0000E3C01FF0E4C020F0216A226AD9CFE9FFB6
:102D1000DACFEAFF1FC00BF020C00CF021C00DF08D
:102D200022C00EF0EECF06F0EECF07F0EECF08F0A7
:102D3000EFCF09F00FEC3EF005C0EDFF04C0EDFF52
:102D400003C0EDFF02C0EFFFD9CFE9FFDACFEAFF02
:102D5000080EE76ED890030EEB32020EEB32010E36
:102D6000EB32EF32E706F6E1D9CFE9FFDACFEAFF3F
:102D7000D880FF0EEE54FF0EEE54000EEE54000EFF
:102D8000EE5406E2DE68DE68DE6ADD6ADD52DD52A0
:102D9000DFCF1FF0010EDBCF20F01FC0F3FF20C0FC
:102DA000F4FF00D0040EE15C02E2E16AE552E16E5C
:102DB000E552E7CFD9FF1200D9CFE6FFE1CFD9FF27
:102DC000020EE126E3C01FF0E4C020F0000ED88020
:102DD0001F56020E20561FC0DEFF20C0DDFFFE0E74
:102DE000DB501F6E206AD9CFE9FFDACFEAFF1FC0A0
:102DF0000DF020C00EF0EECF08F0EDCF09F0F8ECAA
:102E00003CF006C0EEFF07C0EDFFD9CFE9FFDACFF7
:102E1000EAFF080E0F0B06E0EC52D890ED32EF32CD
:102E2000E806FAE1DF5000D01F6E020EE15C02E21C
:102E3000E16AE552E16E1F50E552E7CFD9FF12007B
:102E4000E3C0E6FFE66A1BEC2AF0E552E552E4C077
:102E50001FF0206A1F50E66E010EE66E1BEC2AF092
:102E6000E552E552E5C0E6FF020EE66E1BEC2AF0E5
:102E7000E552E552E6C0E6FF030EE66E1BEC2AF0D3
:102E8000E552E5521200E66A3DEC2AF0E5520001F7
:102E9000E36FE46B010EE66E3DEC2AF0E5521F6E27
:102EA000206A1FC020F01F6A1F500001E327205036
:102EB0000001E423020EE66E3DEC2AF0E55200012B
:102EC000E56F030EE66E3DEC2AF0E5520001E66F79
:102ED00012000001E96B0001EA6B0001EB6BEC6B87
:102EE00012000201E36B0201E46B0201E56BE66B89
:102EF0001200D9CFE6FFE1CFD9FF060EE126DE6A48
:102F0000DD6A020EDB6A030EDB6A040EDB6A050E65
:102F1000DB6A040EDB6A050EDB6A040EDBCF1FF0F2
:102F2000050EDBCF20F0D890205004E6200E1F5C69
:102F3000000E20581EE2040EDBCFE9FF050EDBCFAA
:102F4000EAFF030EEA02F3CFEAFF030EE902F3CF32
:102F5000E9FFF450EA26800EE926020EEA22EF503D
:102F6000DE26000EDD22040EDB2A050E01E3DB2A3D
:102F7000D4D7040EDB6A050EDB6A040EDBCF1FF02C
:102F8000050EDBCF20F0DECF21F0DDCF22F0205088
:102F90002218E8AE02D0223404D021501F5C225007
:102FA00020581EE2040EDB500001F4250F01E96EEB
:102FB000050EDB500001F5210F01EA6EEF501F6E88
:102FC000206AD950020FE96EDACFEAFF1F50EE26D1
:102FD0002050ED22040EDB2A050E01E3DB2ACDD7BB
:102FE000DECF1FF0DDCF20F01F500201406FDECF9B
:102FF0001FF0DDCF20F020C01FF0206A1FC041F27B
:10300000FF0EE76E020EDBCF1FF0030EDBCF20F0CA
:10301000E7501F16206A1FC042F2020EDBCF1FF0DE
:10302000030EDBCF20F020C01FF0206A1FC043F248
:10303000C4EC10F0060EE15C02E2E16AE552E16EDA
:10304000E552E7CFD9FF1200D9CFE6FFE1CFD9FF94
:10305000020EE12686EC3BF0040EE66E60D8E552E7
:10306000C450216E226A21C022F0216AC35000019F
:1030700021241F6E000E2220206E1FC0DEFF20C004
:10308000DDFFDECFE6FFDDCFE6FF24DEE552E552D1
:10309000F3CFDEFFF4CFDDFFDFCF40F2DECF1FF056
:1030A000DDCF20F020C01FF0206A1FC041F2E66A89
:1030B00036D8E552C450216E226A21C022F0216A1E
:1030C000C350000121241F6E000E2220206E1FC05D
:1030D000DEFF20C0DDFFDECFE6FFDDCFE6FFFADD5D
:1030E000E552E552F3CFDEFFF4CFDDFFDFCF42F252
:1030F000DECF1FF0DDCF20F020C01FF0206A1FC000
:1031000043F2C4EC10F071EC3BF0020EE15C02E221
:10311000E16AE552E16EE552E7CFD9FF1200D9CF5F
:10312000E6FFE1CFD9FFFE0EDB28C26EC282C2B23B
:10313000FED7E552E7CFD9FF1200D9CFE6FFE1CFA6
:10314000D9FF020EE126010EEBC0DBFF010EDB50C2
:103150003F0803E2DE523F0EDD6E010EDBCF40F290
:10316000010EDF6E010EDB50D880DF5423E3000137
:10317000EA51EA2BEA6A600FE96E000EEA22EF508C
:10318000E66EDF50EA6A400FE96E020EEA22E5526F
:10319000E750EF6E0001EA511F6E206AD890205070
:1031A00004E6800E1F5C000E205802E30001EA6B6B
:1031B000DF2AD8D7010EDB501F6E206A1F50000196
:1031C000EB5F20500001EC5BC4EC10F0020EE15C00
:1031D00002E2E16AE552E16EE552E7CFD9FF120063
:1031E000D9CFE6FFE1CFD9FF020EE126010EEBC0F9
:1031F000DBFF010EDB50400803E2DE52400EDD6EC5
:10320000DF6A010EDB50DF5C23E20001EA51EA2BAA
:10321000EA6A600FE96E000EEA22EF50E66EDF50B8
:10322000EA6A400FE96E020EEA22E552E750EF6EBD
:103230000001EA511F6E206AD890205004E6800EEB
:103240001F5C000E205802E30001EA6BDF2AD9D789
:10325000010EDB501F6E206A1F500001EB5F2050F3
:103260000001EC5BC4EC10F0020EE15C02E2E16AEA
:10327000E552E16EE552E7CFD9FF1200D9CFE6FF64
:10328000E1CFD9FF200EF36EFE0EDBCFF4FFF3503B
:10329000F45C0DE2FE0EDB50030DF3CFE9FFF4CF3B
:1032A000EAFF800EE926020EEA22EF5003E1000158
:1032B000E88B31D0FE0EDB50030DF3CFE9FFF4CFE6
:1032C000EAFF800EE926020EEA22EF50E66EFE0EBD
:1032D000DB50030DF3CFE9FFF4CFEAFF800EE926C0
:1032E000020EEA22EE5200010001F451EE241F6E9C
:1032F00000010001F551EE20206E1FC0E6FF20C046
:10330000E6FF71DBE552E552E552FD0EDB06FD0EF0
:10331000DB500008CFE3E552E7CFD9FF1200D9CF49
:10332000E6FFE1CFD9FFE652DF6A200EDF5C0DE257
:10333000DF50030DF3CFE9FFF4CFEAFF800EE9265B
:10334000020EEA22EF6ADF2AF0D7E552E552E7CF14
:10335000D9FF1200D9CFE6FFE1CFD9FF040EE12655
:10336000FD0EDBCFE9FFFE0EDBCFEAFFEF50EF2AC9
:10337000EA6A000FE96E020EEA22EF50E66ED950BB
:10338000020FE96EDACFEAFFE552E750EE6EED6A22
:10339000020EDB500201E52500011F6E030EDB501B
:1033A0000201E6210001206E000ED8801F54010E9C
:1033B000205403E20001E88F42D0DE6ADD6ADECFEE
:1033C0001FF0DDCF20F0020EDBCF21F0030EDBCFAC
:1033D00022F021501F5C2250205831E2FD0EDBCF3D
:1033E000E9FFFE0EDBCFEAFFEF50EF2AEA6A000F9B
:1033F000E96E020EEA22EF50E66E0201E351E32B82
:10340000EA6A000FE96E010EEA22E552E750EF6E1C
:103410000201E3511F6E206AD890205004E6000E8E
:103420001F5C010E205802E30201E36B0201E52B51
:10343000000EE623DF2A010E01E3DB2AC0D7040ECB
:10344000E15C02E2E16AE552E16EE552E7CFD9FFC5
:103450001200D9CFE6FFE1CFD9FF080EE126FD0E1D
:10346000DBCFE9FFFE0EDBCFEAFFEF28EA6A000FB1
:10347000E96E020EEA22EFCF1FF0206A1FBE20681D
:10348000040E1FC0DBFF050E20C0DBFF040EDBCFE8
:103490001FF0050EDBCF20F0203404E21F503D0862
:1034A000000E205403E20001E88D4FD2FD0EDBCF69
:1034B000E9FFFE0EDBCFEAFFEF50EA6A000FE96E8C
:1034C000020EEA22EFCF1FF0206A1FBE2068060E10
:1034D0001FC0DBFF070E20C0DBFF020EDB6A030EFE
:1034E000DB6ADE6ADD6ADECF1FF0DDCF20F0D89028
:1034F000205004E6200E1F5C000E205823E2DECF91
:10350000E9FFDDCFEAFF030EEA02F3CFEAFF030E85
:10351000E902F3CFE9FFF450EA26800EE926020E15
:10352000EA22EF501F6E206AD950020FE96EDACFFF
:10353000EAFF1F50EE262050ED22DF2A010E01E3A4
:10354000DB2AD1D7060EDBCFE9FF070EDBCFEAFF80
:10355000030EEA02F3CFEAFF030EE902F3CFE9FF1D
:10356000F450EA26800EE926020EEA22EF501F6E82
:10357000206AD950020FE96EDACFEAFF1F50EE5EE3
:103580002050ED5A040EDBCF1FF0050EDBCF20F0EC
:10359000020EDBCF21F0030EDBCF22F0000ED8802D
:1035A0002156030E225622502018E8AE02D02034B5
:1035B00004D01F50215C2050225803E20001E88D06
:1035C000C4D1060EDBCF1FF0070EDBCF20F0203476
:1035D00004E21F501F08000E205403E20001E88D92
:1035E000B4D1060EDBCFE9FF070EDBCFEAFF030EF7
:1035F000EA02F3CFEAFF030EE902F3CFE9FFF4504A
:10360000EA26800EE926020EEA22EF5001E106D1F9
:10361000060EDBCFE9FF070EDBCFEAFF030EEA025F
:10362000F3CFEAFF030EE902F3CFE9FFF450EA26F5
:10363000800EE926020EEA22EF501F6E206A000E6D
:10364000D8801F56030E20561F06000E205A040E67
:103650001FC0DBFF050E20C0DBFF060EDBCFE9FF3E
:10366000070EDBCFEAFF030EEA02F3CFEAFF030EF9
:10367000E902F3CFE9FFF450EA26800EE926020EB4
:10368000EA22EE52EECFDEFFEDCFDDFFDECF1FF000
:10369000DDCF20F0040EDBCF21F0050EDBCF22F0D2
:1036A00020502218E8AE02D0223404D021501F5CF2
:1036B0002250205835E2060EDBCFE9FF070EDBCFA4
:1036C000EAFF030EEA02F3CFEAFF030EE902F3CFAB
:1036D000E9FFF450EA26800EE926020EEA22EF50B6
:1036E0000001206AF4251F6EF5512022DE501F24B0
:1036F000E96EDD502020EA6EEF50E66EDE500001EC
:10370000F4250F01E96EDD500001F5210F01EA6E8D
:10371000E552E750EF6EDF2A010E01E3DB2AB6D750
:10372000DE6ADD6ADECF1FF0DDCF20F0D8902050BA
:1037300004E6200E1F5C000E205870E2DECFE9FF89
:10374000DDCFEAFF030EEA02F3CFEAFF030EE90240
:10375000F3CFE9FFF450EA26800EE926020EEA22B2
:10376000EECF1FF0EECF20F0EFCF21F0060EDBCF33
:10377000E9FF070EDBCFEAFF030EEA02F3CFEAFF11
:10378000030EE902F3CFE9FFF450EA26800EE926A2
:10379000020EEA22EE52EECF22F0EFCF23F000012C
:1037A00023502118E8AE02D0213404D02050225CEE
:1037B000215023582EE2060EDBCFE9FF070EDBCFA8
:1037C000EAFF030EEA02F3CFEAFF030EE902F3CFAA
:1037D000E9FFF450EA26800EE926020EEA22EF50B5
:1037E0001F6E206ADECFE9FFDDCFEAFF030EEA029B
:1037F000F3CFEAFF030EE902F3CFE9FFF450EA2624
:10380000800EE926020EEA22EE521F50EE5E205094
:10381000ED5ADF2A010E01E3DB2A84D7FD0EDBCF50
:10382000E9FFFE0EDBCFEAFFEF28EA6A000FE96E40
:10383000020EEA22EF50E66E060EDBCFE9FF070E1E
:10384000DBCFEAFF030EEA02F3CFEAFF030EE90241
:10385000F3CFE9FFF450EA26800EE926020EEA22B1
:10386000E552E750EF6E060EDBCFE9FF070EDBCF28
:10387000EAFF030EEA02F3CFEAFF030EE902F3CFF9
:10388000E9FFF450EA26800EE926020EEA22EE5203
:10389000020EDBCFEEFF030EDBCFEDFF020E1F6E3D
:1038A000FD0EDBCFE9FFFE0EDBCFEAFF1F50EF2658
:1038B000DE6ADD6ADECF1FF0DDCF20F0060EDBCF43
:1038C000E9FF070EDBCFEAFF030EEA02F3CFEAFFC0
:1038D000030EE902F3CFE9FFF450EA26800EE92651
:1038E000020EEA22EF50000120AE02D0D89003D0A1
:1038F0001F5C000E205829E2FD0EDBCFE9FFFE0E13
:10390000DBCFEAFFEF50EF2AEA6A000FE96E020E02
:10391000EA22EF50E66E020EDB500001F4250001B2
:103920001F6E030EDB500001F5210001206EDE50FA
:103930001F24E96EDD502020EA6EE552E750EF6E5D
:10394000DF2A010E01E3DB2AB5D7080EE15C02E2B3
:10395000E16AE552E16EE552E7CFD9FF1200F29E2F
:103960006AEC3DF0840EA66EFE0EF66E7F0EF76ECC
:10397000F86AF56A0C00550EA76EAA0EA76EA6820D
:103980004E0EE66E47EC3EF0E552FF001200F00EE0
:103990000001E71781A402D00001E78780AA02D0C6
:1039A0000001E78581B802D00001E78381A602D03B
:1039B0000001E781E7C040F2E8C041F28F0E00014C
:1039C000E7170001E86B8B90C4EC10F012000201C5
:1039D000020E406F02011E0E416F0201010E426F86
:1039E000C4EC10F01200D9CFE6FFE1CFD9FF0D0EE5
:1039F000E126DF6A0B0EDB6A0C0EDB6AF29A070E19
:103A0000D56EFC0EDB5004E0FC0EDB503D0804E2FA
:103A10000001E88B6CEF24F0FE0E0001E81502E0D7
:103A20006CEF24F0FC0EDB50DF5C02E36CEF24F063
:103A3000DF50E76EFD0EDBCFE9FFFE0EDBCFEAFFC6
:103A4000E750E926000EEA22EF50546EB30E545CA4
:103A500004E2FC0EDB50DF6EDFD7D50E545C01E2D2
:103A6000E4D3D50E545E549E5446F9505450F92672
:103A7000C2D3B6D3F9D21BD36BD337D3F1D2E8D2AA
:103A80007ED275D260D257D2FDD12FD2F7D1E2D1FA
:103A9000A9D171D148D15BD103D1F1D0DCD0C3D051
:103AA000AAD081D079D06DD061D049D032D02ED07B
:103AB0002AD026D022D01DD018D014D010D00CD0AF
:103AC00008D004D000D08A98DF2AADD38A88DF2AB4
:103AD000AAD38A86DF2AA7D38A96DF2AA4D38A8428
:103AE000DF2AA1D38A94DF2A9ED30C0EBA6EDF2A76
:103AF0009AD3BA6A8B92DF2A96D3898ADF2A93D324
:103B0000899ADF2A90D38B80DF2A8DD38B90DF2A8E
:103B10008AD3DF2ADF50E76EFD0EDBCFE9FFFE0E12
:103B2000DBCFEAFFE750E926000EEA22EFCFE0F212
:103B3000E0C2E6FF8BEC28F0E552DF2A74D3DF2ADF
:103B4000080EE66EDF50E76EFD0EDBCFE9FFFE0EDE
:103B5000DBCFEAFFE750E926000EEA22EF50E66EDF
:103B60001BEC28F0E552E552DF2A5DD3080EE66E25
:103B7000EBEC27F0E66E1BEC28F0E552E552DF2A6D
:103B800052D3080EE66E6DEC27F0E552E66EB6EC09
:103B900027F0E552DF2A47D3080EE66E6DEC27F0DA
:103BA000E552DF2A40D3DF2ADF50E76EFD0EDBCF80
:103BB000E9FFFE0EDBCFEAFFE750E926000EEA221E
:103BC000EF50E66EDF50E76EFD0EDBCFE9FFFE0E35
:103BD000DBCFEAFFE750E926000EEA22010EE926D4
:103BE000000EEA22EF50E66E1BEC28F0E552E5529B
:103BF000020EDF2618D3DF2ADF50E76EFD0EDBCF83
:103C0000E9FFFE0EDBCFEAFFE750E926000EEA22CD
:103C1000EF50E66EEBEC27F0E66E1BEC28F0E55279
:103C2000E552DF2A00D3DF2ADF50E76EFD0EDBCF3F
:103C3000E9FFFE0EDBCFEAFFE750E926000EEA229D
:103C4000EF50E66E6DEC27F0E552E66EB6EC27F02D
:103C5000E552DF2AE8D2DF2ADF50E76EFD0EDBCF28
:103C6000E9FFFE0EDBCFEAFFE750E926000EEA226D
:103C7000EF50E66E6DEC27F0E552DF2AD4D2DF2A52
:103C8000DF50E76EFD0EDBCFE9FFFE0EDBCFEAFF74
:103C9000E750E926000EEA22EFCFE1F2DF2AC3D295
:103CA0000B0EDB500EE0040EDB06040EDB5005E1CC
:103CB0000B0EDB6A030EDF26B6D2050EDB50DF6E7D
:103CC000B2D2010EF36E0B0EF3CFDBFFDF50E76EC7
:103CD000FD0EDBCFE9FFFE0EDBCFEAFFE750E92662
:103CE000000EEA22010EE926000EEA22EF50DF5C08
:103CF000E76E050EE7CFDBFFDF50E76EFD0EDBCF93
:103D0000E9FFFE0EDBCFEAFFE750E926000EEA22CC
:103D1000020EE926000EEA22040EEFCFDBFF050EAD
:103D2000DB50DF6E80D2DF2ADF50E76EFD0EDBCF87
:103D3000E9FFFE0EDBCFEAFFE750E926000EEA229C
:103D4000EF50E66E05EC27F0E552DF2A6CD2DF2A51
:103D5000DF50E76EFD0EDBCFE9FFFE0EDBCFEAFFA3
:103D6000E750E926000EEA22EF50E66E9BEC24F0C5
:103D7000E552DF2A58D20001E905EA6A600FE96ED0
:103D8000000EEA22010EEFCFDBFFDF50E76EFD0EE3
:103D9000DBCFE9FFFE0EDBCFEAFFE750E926000E9E
:103DA000EA22010EE926000EEA22EF50F36E010E20
:103DB000DB50F35C14E1DF50E76EFD0EDBCFE9FF73
:103DC000FE0EDBCFEAFFE750E926000EEA22020EE4
:103DD000E926000EEA22EF50DF24DF6E02D0030E48
:103DE000DF2621D20001E905EA6A600FE96E000EC4
:103DF000EA22010EEFCFDBFF010EDBCF1FF0DF5019
:103E0000E76EFD0EDBCFE9FFFE0EDBCFEAFFE750EA
:103E1000E926000EEA22010EE926000EEA22EF5002
:103E2000D8801F5414E2DF50E76EFD0EDBCFE9FFB0
:103E3000FE0EDBCFEAFFE750E926000EEA22020E73
:103E4000E926000EEA22EF50DF24DF6E02D0030ED7
:103E5000DF26E9D1DF50E76EFD0EDBCFE9FFFE0E76
:103E6000DBCFEAFFE750E926000EEA22010EE92641
:103E7000000EEA22EF50DF24DF6ED5D1FC0EDB50BE
:103E8000DF6ED1D1DF2ADF50DF2AE76EFD0EDBCFF8
:103E9000E9FFFE0EDBCFEAFFE750E926000EEA223B
:103EA000EF50206A000F1F6E0F0E2022090E1FC058
:103EB000DBFF0A0E20C0DBFFDF50DF2AE76EFD0EBE
:103EC000DBCFE9FFFE0EDBCFEAFFE750E926000E6D
:103ED000EA22EF50E66E090EDBCFE9FF0A0EDBCFD8
:103EE000EAFFE552E750EF6E9ED1DF2ADF50E76E22
:103EF000FD0EDBCFE9FFFE0EDBCFEAFFE750E92640
:103F0000000EEA22EF50206A000F1F6E0F0E2022D3
:103F1000090E1FC0DBFF0A0E20C0DBFF090EDBCF3E
:103F2000E9FF0A0EDBCFEAFFEF50E66EB6EC27F0B2
:103F3000E552DF2A78D1DF2A2CEC25F0E66EB6ECCC
:103F400027F0E55270D1DF2ADF50DF2AE76EFD0E41
:103F5000DBCFE9FFFE0EDBCFEAFFE750E926000EDC
:103F6000EA22EF50E66EAEEC24F0E5525CD1DF2A97
:103F7000EBEC27F0E66EAEEC24F0E55254D10C0EDB
:103F8000DB5016E0070EDB06080E01E2DB06D95017
:103F9000070FE96EDACFEAFFEE50ED1005E10C0EE7
:103FA000DB6A020EDF263FD1060EDB50DF6E3BD10F
:103FB000DF50E76EFD0EDBCFE9FFFE0EDBCFEAFF41
:103FC000E750E926000EEA22010EE926000EEA2259
:103FD000EF50DF5CE76E060EE7CFDBFFEBEC27F080
:103FE000E66ED950070FE96EDACFEAFFE552E750E7
:103FF000EE6EED6AEBEC27F0216E226A086A010E84
:10400000096E21C00DF022C00EF0CBEC3CF006C0D2
:104010001FF007C020F0D950070FE96EDACFEAFF92
:104020001F50EE262050ED22D950070FE96EDACF4F
:10403000EAFFEE50ED1003E1020EDF26F4D0010E90
:10404000F36E0C0EF3CFDBFF060EDB50DF6EEBD012
:10405000ABEC28F0E66EB6EC27F0E552DF2AE3D0B1
:10406000EBEC27F0DF2ADFD0DF2A040EE66E010E2C
:10407000E66E1BEC28F0E552E552080EE66EE66AA5
:104080001BEC28F0E552E552080EE66E24EC27F012
:10409000E552E66EB6EC27F0E552080EE66E24EC2B
:1040A00027F0E552E66EB6EC27F0E552BCD0DF2AE9
:1040B000040EE66EE66A1BEC28F0E552E552080EA7
:1040C000E66EE66A1BEC28F0E552E552080EE66E55
:1040D000E66A1BEC28F0E552E552080EE66EE66A49
:1040E0001BEC28F0E552E5529ED0DF2A040EE66E66
:1040F000E66A1BEC28F0E552E552080EE66EDF504A
:10410000DF2AE76EFD0EDBCFE9FFFE0EDBCFEAFF15
:10411000E750E926000EEA22EF50E66E1BEC28F08D
:10412000E552E552080EE66EDF50DF2AE76EFD0E1F
:10413000DBCFE9FFFE0EDBCFEAFFE750E926000EFA
:10414000EA22EF50E66E1BEC28F0E552E5526BD008
:10415000DF2A040EE66EE66A1BEC28F0E552E55213
:10416000080EE66EDF50DF2AE76EFD0EDBCFE9FFBB
:10417000FE0EDBCFEAFFE750E926000EEA22EF5001
:10418000E66E1BEC28F0E552E552080EE66EDF50B5
:10419000DF2AE76EFD0EDBCFE9FFFE0EDBCFEAFF85
:1041A000E750E926000EEA22EF50E66E1BEC28F0FD
:1041B000E552E552080EE66EDF50DF2AE76EFD0E8F
:1041C000DBCFE9FFFE0EDBCFEAFFE750E926000E6A
:1041D000EA22EF50E66E1BEC28F0E552E55223D0C0
:1041E000DF2A080EE66E24EC27F0E552E66EB6EC08
:1041F00027F0E55218D0DF2ADF50E76EFD0EDBCF47
:10420000E9FFFE0EDBCFEAFFE750E926000EEA22C7
:10421000EF50E66E24EC27F0E552E66EB6EC27F0A0
:10422000E552DF2A00D00CEF1DF0B30E545E549E11
:104230005446F9505450F92680D287D241D3DED269
:104240002FD3E0D28BD265D250D227D2EBD1C0D1BE
:1042500098D190D17CD174D167D14ED143D13AD18C
:1042600025D119D10ED105D1F0D0EBD0E6D0DDD0DB
:10427000C6D0ADD084D070D001D036D0DF2A040EA5
:10428000E66EE66A1BEC28F0E552E552040EE66E97
:10429000DF50E76EFD0EDBCFE9FFFE0EDBCFEAFF5E
:1042A000E750E926000EEA22EF50E66E1BEC28F0FC
:1042B000E552E552080EE66EEBEC27F0E66E1BECDD
:1042C00028F0E552E552080EE66EE66A1BEC28F08F
:1042D000E552E552040EE66E020EE66E1BEC28F087
:1042E000E552E552DF2A9FD7DF2A040EE66EE66A22
:1042F0001BEC28F0E552E552040EE66EDF50E76E47
:10430000FD0EDBCFE9FFFE0EDBCFEAFFE750E9262B
:10431000000EEA22EF50E66E1BEC28F0E552E55263
:10432000080EE66EEBEC27F0E66E1BEC28F0E5528B
:10433000E552080EE66EEBEC27F0E66E1BEC28F07B
:10434000E552E552040EE66E020EE66E1BEC28F016
:10435000E552E552DF2A67D7DF2ADF50E76EFD0E10
:10436000DBCFE9FFFE0EDBCFEAFFE750E926000EC8
:10437000EA22EF50E66EBADAE552DF2A54D7DF2A96
:10438000DF50E76EFD0EDBCFE9FFFE0EDBCFEAFF6D
:10439000E750E926000EEA22EF50E66EDF50E76EA6
:1043A000FD0EDBCFE9FFFE0EDBCFEAFFE750E9268B
:1043B000000EEA22010EE926000EEA22EF50E66E18
:1043C00053EC28F0E552E552020EDF262CD7DF2A07
:1043D000DF50E76EFD0EDBCFE9FFFE0EDBCFEAFF1D
:1043E000E750E926000EEA22EF50E66EEBEC27F0EC
:1043F000E66E53EC28F0E552E552DF2A14D7DF2AA7
:10440000DF50E76EFD0EDBCFE9FFFE0EDBCFEAFFEC
:10441000E750E926000EEA22EFCFE2F2E2C2E6FF21
:10442000BEEC28F0E552DF2AFED6D2EC28F0E66E8C
:10443000B6EC27F0E552DF2AF6D6E3EC28F0DF2AC7
:10444000F2D6F8EC28F0DF2AEED6DF2ADF50E76E4E
:10445000FD0EDBCFE9FFFE0EDBCFEAFFE750E926DA
:10446000000EEA22EF50E66E0DEC29F0E552DF2A4D
:10447000DAD6DF2AEBEC27F0E66E0DEC29F0E552F8
:10448000D2D6E66A76EC29F0E552E66EB6EC27F075
:10449000E552DF2AC8D60F0EE66E76EC29F0E5521B
:1044A000E66EB6EC27F0E552DF2ABDD6DF2ADF50F4
:1044B000E76EFD0EDBCFE9FFFE0EDBCFEAFFE75034
:1044C000E926000EEA22EF50E66EDDEC29F0E55217
:1044D000DF2AA9D6DF2AEBEC27F0E66EDDEC29F027
:1044E000E552A1D6E66ADDEC29F0E552E66EB6ECBF
:1044F00027F0E552DF2A97D6DF2ADF50E76EFD0E60
:10450000DBCFE9FFFE0EDBCFEAFFE750E926000E26
:10451000EA22EF50E66EDDEC29F0E552E66EB6ECED
:1045200027F0E552DF2A7FD6DF2AEBEC27F0E66E94
:10453000DDEC29F0E552E66EB6EC27F0E55273D6D5
:10454000DF2A83DBE66EB6EC27F0E5526CD6DF2A75
:10455000DF50DF2AE76EFD0EDBCFE9FFFE0EDBCF7B
:10456000EAFFE750E926000EEA22EF50E66EE5DAB0
:10457000E55259D6DF2AEBEC27F0E66EDEDAE5529B
:1045800052D6DF2AD5DB020EF3CFDBFF030EF4CFCA
:10459000DBFFFF0EE76E020EDBCF1FF0030EDBCF5B
:1045A00020F0E7501F16206A1F50E66EB6EC27F089
:1045B000E552020EDBCF1FF0030EDBCF20F020C050
:1045C0001FF0206A1F50E66EB6EC27F0E5522BD69E
:1045D000DF2AE66ADF50E76EFD0EDBCFE9FFFE0E55
:1045E000DBCFEAFFE750E926000EEA22010EE926BA
:1045F000000EEA22EF50E66EDF50E76EFD0EDBCFD5
:10460000E9FFFE0EDBCFEAFFE750E926000EEA22C3
:10461000EF50E66E4CEC2AF0E552E552E552020E00
:10462000DF2601D6DF2ADF50E76EFD0EDBCFE9FF84
:10463000FE0EDBCFEAFFE750E926000EEA22020E6B
:10464000E926000EEA22EF50E66EDF50E76EFD0E1F
:10465000DBCFE9FFFE0EDBCFEAFFE750E926000ED5
:10466000EA22010EE926000EEA22EF50E66EDF5044
:10467000E76EFD0EDBCFE9FFFE0EDBCFEAFFE75072
:10468000E926000EEA22EF50E66E4CEC2AF0E552E5
:10469000E552E552030EDF26C6D5DF2ADF50E76E6E
:1046A000FD0EDBCFE9FFFE0EDBCFEAFFE750E92688
:1046B000000EEA22010EE926000EEA22EF50E66E15
:1046C000DF50E76EFD0EDBCFE9FFFE0EDBCFEAFF2A
:1046D000E750E926000EEA22EF50E66EA1EC2BF03F
:1046E000E552E552020EDF269ED5DF2ADF50E76E47
:1046F000FD0EDBCFE9FFFE0EDBCFEAFFE750E92638
:10470000000EEA22EF50E66EE5EC2BF0E552DF2AD0
:104710008AD5DF2ADF50E76EFD0EDBCFE9FFFE0E04
:10472000DBCFEAFFE750E926000EEA22EF50E66E03
:1047300006EC2CF0E552DF2A76D5DF2AE66AE66A37
:1047400069EC2DF0E552E5526ED5DF2A010EE66EDA
:10475000E66A69EC2DF0E552E55265D5DF2A010ED7
:10476000E66EDF50E76EFD0EDBCFE9FFFE0EDBCF1E
:10477000EAFFE750E926000EEA22EF50E66EDF502E
:10478000E76EFD0EDBCFE9FFFE0EDBCFEAFFE75061
:10479000E926000EEA22010EE926000EEA22EF5079
:1047A000E66EDF50E76EFD0EDBCFE9FFFE0EDBCFDE
:1047B000EAFFE750E926000EEA22020EE926000E83
:1047C000EA22EF50E66EDF50E76EFD0EDBCFE9FF29
:1047D000FE0EDBCFEAFFE750E926000EEA22030EC9
:1047E000E926000EEA22EF50E66E36EC2CF01F6E42
:1047F000050EE15E1F50040EDF2615D5DF2A18ECEA
:104800002DF011D5DF2ADF50E76EFD0EDBCFE9FF7B
:10481000FE0EDBCFEAFFE750E926000EEA22EF505A
:10482000E66EDF50E76EFD0EDBCFE9FFFE0EDBCF5D
:10483000EAFFE750E926000EEA22010EE926000E03
:10484000EA22EF50E66EDF50E76EFD0EDBCFE9FFA8
:10485000FE0EDBCFEAFFE750E926000EEA22020E49
:10486000E926000EEA22EF50E66EDF50E76EFD0EFD
:10487000DBCFE9FFFE0EDBCFEAFFE750E926000EB3
:10488000EA22030EE926000EEA22EF50E66EC7EC9C
:104890002CF0E552E552E552E552040EDF26C3D472
:1048A000DF2A99DBE66E97DBE66E95DBE66E93DB3F
:1048B000E66EC7EC2CF0E552E552E552E552B3D472
:1048C000DF2A010EE66E010EE66E69EC2DF0E55270
:1048D000E552A9D40CEF1DF00D0EE15C02E2E16A95
:1048E000E552E16EE552E7CFD9FF1200D9CFE6FFDE
:1048F000E1CFD9FF0201E351E32BEA6A000FE96E31
:10490000010EEA22FE0EDBCFEFFF0201E3511F6E24
:10491000206AD890205004E6000E1F5C010E20583B
:1049200002E30201E36B0201E52B000EE623E552F0
:10493000E7CFD9FF1200D9CFE6FFE1CFD9FFF2943C
:10494000FE0EDB50FF0DF350D76ED66AD58EF2A463
:10495000FED7D59EE552E7CFD9FF1200D9CFE6FFAB
:10496000E1CFD9FFF29ECD90A40ED76E730ED66E16
:10497000F294D58E8050080B04E1F250040B01E153
:10498000F9D7F2B45DD089949294600EE66E80EC13
:104990003EF0E55289848050080B04E0F250040B8D
:1049A00001E1F9D7F2B44CD0FE0EDB50546EF2B6F2
:1049B00046D080A6FCD7899454BE898480B6FED7A1
:1049C000F2B63DD080A6FCD7899454BC898480B6C9
:1049D000FED7F2B634D080A6FCD7899454BA898425
:1049E00080B6FED7F2B62BD080A6FCD7899454B8F7
:1049F000898480B6FED7F2B622D080A6FCD78994EF
:104A000054B6898480B6FED7F2B619D080A6FCD7FA
:104A1000899454B4898480B6FED7F2B610D080A6AB
:104A2000FCD7899454B2898480B6FED7F2B607D0F9
:104A300080A6FCD7899454B0898480B6FED7000044
:104A4000F2A402D00001E885D59EF28ECD8000D080
:104A5000E552E7CFD9FF1200CD90F29EA40ED76E9B
:104A6000730ED66EF294D58E8050080B04E1F2508E
:104A7000040B01E1F9D7F2B454D089949294600EFA
:104A8000E66E80EC3EF0E55289848050080B04E02D
:104A9000F250040B01E1F9D79284F2B442D0546A87
:104AA000F2B63ED080A6FCD780B6FED780B4548E36
:104AB000F2B636D080A6FCD780B6FED780B4548C30
:104AC000F2B62ED080A6FCD780B6FED780B4548A2A
:104AD000F2B626D080A6FCD780B6FED780B4548824
:104AE000F2B61ED080A6FCD780B6FED780B454861E
:104AF000F2B616D080A6FCD780B6FED780B4548418
:104B0000F2B60ED080A6FCD780B6FED780B4548211
:104B1000F2B606D080A6FCD780B6FED780B454800B
:104B2000000089849294F2A402D00001E885D59E09
:104B3000F28ECD80545000D01200D9CFE6FFE1CFE5
:104B4000D9FFF29ECD90A40ED76E730ED66EF2945E
:104B5000D58E92848050040B04E0F250040B01E1E6
:104B6000F9D7F2B45FD092968986600EE66E80EC3B
:104B70003EF0E55289968050040B04E1F250040B9C
:104B800001E1F9D792869294F2B44CD0FE0EDB503C
:104B9000546EF2B646D080A6FCD7899454BE898460
:104BA00080B6FED7F2B63DD080A6FCD7899454BC1F
:104BB000898480B6FED7F2B634D080A6FCD789941B
:104BC00054BA898480B6FED7F2B62BD080A6FCD723
:104BD000899454B8898480B6FED7F2B622D080A6D4
:104BE000FCD7899454B6898480B6FED7F2B619D022
:104BF00080A6FCD7899454B4898480B6FED7F2B6D7
:104C000010D080A6FCD7899454B2898480B6FED790
:104C1000F2B607D080A6FCD7899454B0898480B6B8
:104C2000FED70000F2A402D00001E885600EE66E17
:104C300080EC3EF0E552D59EF28ECD809284929625
:104C400000D0E552E7CFD9FF1200CD90F29EA40E1E
:104C5000D76E730ED66EF294D58E92848050040B6C
:104C600004E0F250040B01E1F9D7F2B455D092966A
:104C70008986600EE66E80EC3EF0E55289968050A3
:104C8000040B04E1F250040B01E1F9D792849286FF
:104C9000F2B442D0546AF2B63ED080A6FCD780B6B9
:104CA000FED780B4548EF2B636D080A6FCD780B63C
:104CB000FED780B4548CF2B62ED080A6FCD780B636
:104CC000FED780B4548AF2B626D080A6FCD780B630
:104CD000FED780B45488F2B61ED080A6FCD780B62A
:104CE000FED780B45486F2B616D080A6FCD780B624
:104CF000FED780B45484F2B60ED080A6FCD780B61E
:104D0000FED780B45482F2B606D080A6FCD780B617
:104D1000FED780B454800000F2A402D00001E885E0
:104D2000D59E92849296F28ECD80545000D012007F
:104D3000D9CFE6FFE1CFD9FF030EE126DF6AF29477
:104D4000800ED76ED66AD58EF2AE02D0010EDF6E1F
:104D5000F29E80A40AD0F2A407D0D59EDF0401E120
:104D6000F28EF36AF46A47D0F4D780B40AD0F2A482
:104D700007D0D59EDF0401E1F28EF36AF46A3BD0DE
:104D8000F4D7800ED76ED66AF29480A40AD0F2A42B
:104D900007D0D59EDF0401E1F28EF368F4682BD0D2
:104DA000F4D7D59EDF0401E1F28ED650E66ED950DD
:104DB000010FE96EDACFEAFFE552E750EE6EED6AD9
:104DC0007F0ED7141F6E206A1FC020F01F6AD950B3
:104DD000010FE96EDACFEAFF1F50EE262050ED22D8
:104DE000010EDBCF1FF0020EDBCF20F01FC0F3FF60
:104DF00020C0F4FF00D0030EE15C02E2E16AE5525C
:104E0000E16EE552E7CFD9FF1200D9CFE6FFE1CF3F
:104E1000D9FFF294D768080EE66E8EEC3EF0E552AC
:104E2000FE0EDB0402E10CD002D0FE0EDB06FE0E0D
:104E3000DB50FF0DF350D66ED58EF2A4FED7D59E73
:104E4000E552E7CFD9FF1200D9CFE6FFE1CFD9FF76
:104E5000E6529284546AFE0EDB50556E020E020139
:104E6000E15D0CE280B454808986000000000000FF
:104E7000899600005442552EF5D718D00201E1055D
:104E8000566E565080B454808986000000000000A1
:104E900000000000E82EFBD7899656500000000065
:104EA0000000E82EFBD75442552EEBD7FE0EDBCF89
:104EB000E6FF080EE552D880E754070B04E05442A1
:104EC000549EE806FCE10201E0A39294545000D005
:104ED000E552E552E7CFD9FF1200D9CFE6FFE1CF87
:104EE000D9FFE6529284546AFE0EDB50556E020ED4
:104EF0000201E15D0CE2898600000000000080B440
:104F00005480899600005442552EF5D718D00201DE
:104F1000E105566E89860000000056500000000032
:104F20000000E82EFBD780B45480899656500000CC
:104F300000000000E82EFBD75442552EEBD7FE0EA2
:104F4000DBCFE6FF080EE552D880E754070B04E0FC
:104F50005442549EE806FCE10201E0A392945450AE
:104F600000D0E552E552E7CFD9FF1200D9CFE6FFD6
:104F7000E1CFD9FF010E0001206AEB251F6EEC5135
:104F80002022800ED8801F54000E205403E200011E
:104F9000E8871DD00001E951E92BEA6A600FE96E4C
:104FA000000EEA22FE0EDBCFEFFF0001E9511F6E7B
:104FB000206AD890205004E6800E1F5C000E205816
:104FC00002E30001E96B0001EB2B000EEC23E5523C
:104FD000E7CFD9FF1200D9CFE6FFE1CFD9FFE652E4
:104FE0000201E551E61104E10001E889000E1ED03E
:104FF0000201E451E42BEA6A000FE96E010EEA2295
:10500000EFCFDFFF0201E507000EE65B0201E4518E
:105010001F6E206AD890205004E6000E1F5C010E1F
:10502000205802E30201E46BDF5000D0E552E55264
:10503000E7CFD9FF1200D9CFE6FFE1CFD9FFE65283
:10504000FE0EDB50546EFD0EDB50556E020E02015B
:10505000E15D0CE254A0899454B0898400008986F3
:10506000000089965442552EF5D718D00201E1056B
:10507000566E54A0899454B08984565000000000A4
:105080000000E82EFBD78986565000000000000083
:10509000E82EFBD789965442552EEBD7E552E552C0
:1050A000E7CFD9FF1200D9CFE6FFE1CFD9FFE65213
:1050B000FE0EDB50546EFD0EDB50556E020E0201EB
:1050C000E15D0CE254A0899454B089848986000083
:1050D000899600005442552EF5D718D00201E105FB
:1050E000566E54A0899454B0898456508986000025
:1050F00000000000E82EFBD7899656500000000003
:105100000000E82EFBD75442552EEBD7E552E5526E
:10511000E7CFD9FF1200D9CFE6FFE1CFD9FFFE0ECE
:10512000DBA402D0898601D08996FE0EDBA602D0D0
:10513000898401D08994FE0EDBA002D0928601D032
:105140009296FE0EDBA202D0928401D09294E55298
:10515000E7CFD9FF1200D9CFE6FFE1CFD9FFE65262
:10516000DF6A80B4DF8280A602D0000EDB80DF50D1
:1051700000D0E552E552E7CFD9FF1200D9CFE6FFC4
:10518000E1CFD9FFFE0EDBA202D0898801D0899839
:10519000FE0EDBA002D0928801D09298E552E7CFB4
:1051A000D9FF1200D9CFE6FFE1CFD9FFE652DF6A7F
:1051B00080A802D0000EDB80DF5000D0E552E5521F
:1051C000E7CFD9FF12008986060EE66E8EEC3EF020
:1051D000E55289989298060EE66E8EEC3EF0E55206
:1051E0008996060EE66E8EEC3EF0E552928812002D
:1051F0008996060EE66E8EEC3EF0E55289989298FE
:10520000060EE66E8EEC3EF0E5528986060EE66EE0
:105210008EEC3EF0E55292881200D9CFE6FFE1CF46
:10522000D9FFFE0EDB50546E080E556E8998020EA3
:105230000201E15D23E254AE929854BE928800D000
:1052400000D000D08986000000D000D000D000D06F
:105250008996000000D000D05446552EECD7928895
:1052600000D000D000D000D000D08986000000D04F
:1052700000D000D080B8558089962FD00201E1512E
:10528000E824FF0F566E54AE929854BE9288565042
:10529000000000D000D000D0E82EFAD78986565002
:1052A00000D000D000D0E82EFDD7899600005446EB
:1052B000552EE9D79288565000D000D0000000D07B
:1052C00000D000D0E82EFAD78986565000D000D002
:1052D000E82EFDD780B8558089965550000802E227
:1052E0000001E885E552E7CFD9FF1200D9CFE6FFEC
:1052F000E1CFD9FF546A080E556E010E566E9288A2
:10530000020E0201E15D14E2544600D000D000D04C
:1053100000D00000898600D000D000D0000080B806
:105320005480899600D000D000D0552EEDD725D0DE
:105330000201E151E824FF0F566E5446000000D0F0
:10534000565000D000D000D00000E82EFAD7898651
:10535000565000D000D0E82EFDD780B854808996F2
:1053600000D0552EEAD70000565000D000D000D013
:1053700000D000D00000E82EFAD78998FE0EDB504E
:1053800001E19298565000D000D000D000D000D05B
:105390000000E82EFAD78986565000D000D0E82EBB
:1053A000FDD700D0899600D00000000092885450AC
:1053B00000D0E552E7CFD9FF1200D9CFE6FFE1CF09
:1053C000D9FFE652FE0EDB50546E080E556E020EEB
:1053D0000201E15D0DE254AE899854BE8988898648
:1053E0005446549080B454808996552EF4D71BD0DF
:1053F0000201E105566E54AE899854BE8988565014
:10540000000000000000E82EFBD789865446549027
:1054100080B454805650000000000000E82EFBD7F6
:105420008996552EE8D78998545000D0E552E55218
:10543000E7CFD9FF1200D9CFE6FFE1CFD9FFE6527F
:10544000DF6AFE0EDB50A96EFD0EDB50A86EA66A69
:10545000A684F2AE02D0010EDF6EF29E550EA76E4C
:10546000AA0EA76EA682DF0401E1F28EA6B2FED7D5
:10547000E552E552E7CFD9FF1200D9CFE6FFE1CFE1
:10548000D9FFFE0EDB50A96EA66AA680A85000D0F8
:10549000E552E7CFD9FF1200D9CFE6FFE1CFD9FF20
:1054A000040EE126DF6A010EDB6A0201E151010808
:1054B00008E2120E566E0F0EF36E030EF3CFDBFFF3
:1054C00007D0C60E566E030EF36E030EF3CFDBFF4E
:1054D00089889298180EE66E8EEC3EF0E552020E28
:1054E0001F6EFD0EDBCFE7FF1F50E726FD0EE7CF57
:1054F000DBFF480ED56E550E546E8998D66AF2942D
:10550000D58EF2AE02D0010EDF6EF29EFD0EDB06EE
:10551000020EDB6A020EDBCF1FF0080EE76E1F18CB
:10552000E8AE02D0E73402D0E7501F5C21E2895098
:10553000EF0B54AE1009F2A4FED7896E5650D62652
:105540009298F294549E54468950556EFD0EDB504D
:1055500005E1FC0EDB5002E1558801D05598F2A41C
:10556000FED789785650D626F294020EDB2AD2D77F
:105570005550F2A4FED7896E5650D626F294010EED
:10558000DB5007E0FD0EDB50000803E224DD546E23
:1055900003D0FE0EDB50546EF2A4FED7897856502D
:1055A000D626F294F2A4FED792885650D626F294CC
:1055B000030EDBCFE6FF8EEC3EF0E552010EDB5032
:1055C00009E08050100B06E00001E885FD0EDB6A63
:1055D000FC0EDB6AF2A4FED700005650D626F294E9
:1055E000030EDBCFE6FF8EEC3EF0E552010EDB5002
:1055F00009E08050100B06E10001E885FD0EDB6A32
:10560000FC0EDB6ADE52010EDD6EFD0EDB50000883
:1056100001E27CD7FC0EDBCFF3FFDB06F350000882
:1056200001E37FD0546A020EDB6A020EDBCF1FF06B
:10563000080EE76E1F18E8AE02D0E73402D0E7503C
:105640001F5C30E2F2A4FED70000D66AF2948950C3
:10565000556EFC0EDB5002E1558801D05598030EC3
:10566000DB04E66E8EEC3EF0E55280B807D0F2B473
:1056700002D080A8FCD75650D66E06D0F2B402D025
:1056800080B8FCD75650D66EF294030EDBCFE6FFFF
:105690008EEC3EF0E552549E544680B8542A020ED9
:1056A000DB2AC3D75550F2A4FED7896E5650D626B2
:1056B0009298F2945450E66E59DCE552F2A4FED76B
:1056C00089785650D626F294F2A4FED79288565086
:1056D000D626F294030EDBCFE6FF8EEC3EF0E552C9
:1056E000010EDB5007E08050100B04E00001E8855C
:1056F000FC0EDB6AF2A4FED700005650D626F294C8
:10570000030EDBCFE6FF8EEC3EF0E552010EDB50E0
:1057100007E08050100B04E10001E885FC0EDB6A15
:1057200079D7DF0401E1F28E070ED56E9288040E60
:10573000E15C02E2E16AE552E16EE552E7CFD9FFB2
:105740001200D9CFE6FFE1CFD9FFE652FE0EDB50C3
:1057500001E10FD0546AFD0EDB50556EDF6AFE0E7C
:10576000DB50DF5C06E225EC38F055905542DF2A2D
:10577000F6D7E552E552E7CFD9FF1200D9CFE6FFC1
:10578000E1CFD9FFE652FE0EDB5002E1000E18D049
:10579000FD0EDB50546EFC0EDB50556E566ADF6A10
:1057A000FE0EDB50DF5C0AE25690564225EC38F0E4
:1057B0005490544255905542DF2AF2D7565000D0AB
:1057C000E552E552E7CFD9FF1200D9CFE6FFE1CF8E
:1057D000D9FF030EE66E040EE66EB3DFE552E55226
:1057E000100EE66EFE0EDBCFE6FF050EE66EC6DFA0
:1057F000E552E552E552010EE66E020EE66EA1DFBD
:10580000E552E552E552E7CFD9FF1200D9CFE6FFC6
:10581000E1CFD9FFE652DF6A010EE66E030EE66EB7
:1058200090DFE552E55256AE02D0010EDF6E800EDB
:10583000E66EFE0EDBCFE6FF080EE66E9FDFE5525A
:10584000E552E5525650E824DF12DFCFE6FFB6EC12
:1058500027F0E552010EE66E020EE66E72DFE552AB
:10586000E552E552E552E7CFD9FF1200D9CFE6FF66
:10587000E1CFD9FF020EE126DF6A010EDB6A010EDD
:10588000E66E030EE66E5DDFE552E55256AE02D0DF
:10589000010EDF6EE66AFB0EDBCFE6FF080EE66E5A
:1058A0006DDFE552E552E5525650E824DF12FA0E5C
:1058B000DB5005E0DFCFE6FFB6EC27F0E552DF6A0C
:1058C00056AE02D0010EDF6EE66AFC0EDBCFE6FFBD
:1058D000080EE66E53DFE552E552E5525650E824D5
:1058E000DF12FA0EDB5005E0DFCFE6FFB6EC27F063
:1058F000E552DF6A56AE02D0010EDF6EE66AFD0E9B
:10590000DBCFE6FF080EE66E39DFE552E552E552E1
:105910005650E824DF12FA0EDB5005E0DFCFE6FF39
:10592000B6EC27F0E552010EDFCFDBFFDF6A56AEA3
:1059300002D0010EDF6E800EE66EFE0EDBCFE6FFBC
:10594000080EE66E1BDFE552E552E5525650E8249C
:10595000DF12FA0EDB5005E0DFCFE6FFB6EC27F0F2
:10596000E552010EE66E020EE66EEBDEE552E55202
:10597000010EDB5000D01F6E020EE15C02E2E16A14
:10598000E552E16E1F50E552E7CFD9FF1200D9CFA3
:10599000E6FFE1CFD9FF010EE66E030EE66ED1DE23
:1059A000E552E55256BE0AD01F0EE66E050EE66EB3
:1059B000C8DEE552E5520001E88536D0E66A010E00
:1059C000E66EBFDEE552E552E66AFB0EDBCFE6FF90
:1059D000080EE66ED3DEE552E552E552E66AFC0EAD
:1059E000DBCFE6FF080EE66EC9DEE552E552E55272
:1059F000E66AFD0EDBCFE6FF080EE66EBFDEE5527F
:105A0000E552E552800EE66EFE0EDBCFE6FF080E95
:105A1000E66EB4DEE552E552E552010EE66E020E88
:105A2000E66E8FDEE552E552E552E7CFD9FF120070
:105A3000D9CFE6FFE1CFD9FFE652D76AD66AF29412
:105A4000D58E0A0EE66EC1DEE552E66AE66AD00E33
:105A5000E66E040EE66EE66A09DF1F6E050EE15E75
:105A60001F50DF6E040EDF1403E1F250040BEDE073
:105A7000F2A404D00001E885D59E26D0090EE66E7A
:105A8000A4DEE552E66AEBEC27F0E66EEBEC27F0DD
:105A9000E66EEBEC27F0E66EEBEC27F0E66EE6DE6A
:105AA0001F6E050EE15E1F500A0EE66E8EDEE55299
:105AB000E66AE66AC00EE66EE66AE66AD7DE1F6E42
:105AC000050EE15E1F50D59EE552E552E7CFD9FFA6
:105AD0001200D9CFE6FFE1CFD9FFE652D76AD66AE6
:105AE000F294D58E0A0EE66E70DEE552E66AE66A3C
:105AF000D00EE66E040EE66EE66AB8DE1F6E050E88
:105B0000E15E1F50DF6E040EDF1403E1F250040B60
:105B1000EDE0F2A404D00001E885D59E23D0090E63
:105B2000E66E53DEE552FE0EDBCFE6FFE66AE66A7E
:105B3000E66AE66A9BDE1F6E050EE15E1F50FD0EF3
:105B4000DB500FE00A0EE66E40DEE552E66AE66ADA
:105B5000C00EE66EE66AE66A89DE1F6E050EE15E3D
:105B60001F50D59EE552E552E7CFD9FF1200D9CF9D
:105B7000E6FFE1CFD9FF020EE126F29E86EC3BF074
:105B80009284928692888FEC19F08B80E950DF6EB8
:105B9000010EEACFDBFF5F5002E05F6A02D058508F
:105BA0005F6E3BEC38F05E50000803E2C3EC38F067
:105BB00007D05F5003E088EC38F002D04DEC38F0AD
:105BC000DF50E96E010EDB50EA6E8B9071EC3BF01A
:105BD000F28E54C040F255C041F2C4EC10F0020EF7
:105BE000E15C02E2E16AE552E16EE552E7CFD9FFFE
:105BF00012000100347D0000F400000002000000EB
:105C0000D9CFE6FFE1CFD9FFE6520401B06B040122
:105C1000B16BB26B196AC56AC76A280EC66E1F0ED1
:105C2000C86EC584C5B4FED7E552E552E7CFD9FFAB
:105C30001200D9CFE6FFE1CFD9FFE6528B9C67D89F
:105C40000401B06B9E960401B051B02BEA6AC00FFC
:105C5000E96E040EEA22EF50C96E9EA6FED7C5BCBF
:105C6000C584400E0401B05DEDE3C584C5B4FED724
:105C7000060EE66E47EC3EF0E5520401B06B0401FF
:105C8000B12B000EB2238B8CE552E552E7CFD9FF42
:105C90001200D9CFE6FFE1CFD9FFE65238D801098B
:105CA000DF6EC582C5B2FED79E96DF50C96E9EA636
:105CB000FED7C5BCC5840401B06B9E96C5869EA662
:105CC000FED70401B051B02BEA6AC00FE96E040E92
:105CD000EA22C9CFEFFF400E0401B05D02E1C58AA0
:105CE00001D0C59AC588C5B8FED7400E0401B05D85
:105CF000E4E3C584C5B4FED70401B06B0401B12B45
:105D0000000EB223E552E552E7CFD9FF1200D9CFFA
:105D1000E6FFE1CFD9FF020EE126DE52A00EDD6ED6
:105D20001D5007E10401B251040B02E0010EDB82B9
:105D30000CD00401B251080B02E0010EDB82040119
:105D4000B251040B02E0010EDB86C580C5B0FED760
:105D50009E96010EDB50C96EB1C41FF0B2C420F094
:105D6000D89020321F32D89020321F321F50DF6E61
:105D70009EA6FED7C5BCC5849E96DF50C96EB1C431
:105D80001FF0B2C420F0060ED8901F362036E8046B
:105D9000FBE11F50DF6E9EA6FED7C5BCC5849E9654
:105DA000DF50C96E9EA6FED7C5BCC584010EDB5070
:105DB00000D01F6E020EE15C02E2E16AE552E16E84
:105DC0001F50E552E7CFD9FF1200D9CFE6FFE1CF50
:105DD000D9FF0401B051B02BEA6AC00FE96E040E7E
:105DE000EA22FE0EDBCFEFFF0401B0513F0801E2D3
:105DF00020DFE552E7CFD9FF12000401B0513F0880
:105E000003E247DF0401B06B0401B051B02BEA6A32
:105E1000C00FE96E040EEA22EF5000D01200D9CF75
:105E2000E6FFE1CFD9FF1E6AFE0EDBCFE6FF0BD8FF
:105E3000E552000904E0010E1E6EE2DE8B80E552A1
:105E4000E7CFD9FF1200D9CFE6FFE1CFD9FFFE0E91
:105E5000DBCFF3FFDB2AF350EA6A000FE96E020E94
:105E6000EA22EF50500802E0000E20D0FE0EDBCFF9
:105E7000F3FFDB2AF350EA6A000FE96E020EEA2212
:105E8000EF504B0802E0000E11D0FE0EDBCFF3FF07
:105E9000DB2AF350EA6A000FE96E020EEA22EF50A5
:105EA000320802E0000E02D0010E00D0E552E7CF2A
:105EB000D9FF1200AD0EE66E88DFE5520401B05145
:105EC0000008F8E31E6A8B901200D9CFE6FFE1CFFD
:105ED000D9FF020EE126DF6A010EDB6ADF50EA6AB3
:105EE000000FE96E020EEA22EF50840A01E14ED162
:105EF000210A01E129D1270A01E126D1010A01E1A4
:105F000023D1040A01E120D1070A01E11DD1010AD0
:105F100001E11AD1230A01E115D1010A01E112D1EF
:105F20000D0A01E10FD1010A01E10CD1080A01E1DA
:105F3000FDD00E0A01E1FAD0030A01E1F7D0010A0F
:105F400001E1F4D0070A01E1F1D0290A01E1EED024
:105F5000030A01E1EBD02E0A01E1BCD00E0A01E1F7
:105F60008DD0020A54E0140A4FE0100A20E0010A22
:105F70001EE0130A19E0030A0CE0070A06E01B0AF8
:105F800001E03CD1400EDF6E3AD1400EDF6E92DF71
:105F900036D1020EDF26DF50EA6A000FE96E020EEC
:105FA000EA22EF28DF262BD1030EDF2628D1DF508F
:105FB000DF2AEA6A000FE96E020EEA22EF50E66E6F
:105FC00004DFE552DF50DF2AEA6A000FE96E020EB5
:105FD000EA22EF50E66EF9DEE552DF50DF2AEA6A88
:105FE000000FE96E020EEA22EF50E66EEEDEE55299
:105FF000DF50DF2AEA6A000FE96E020EEA22EF5054
:10600000E66EE3DEE552FBD0050EDF26F8D0DF506A
:10601000DF2AEA6A000FE96E020EEA22EF50E66E0E
:10602000D4DEE552DF50DF2AEA6A000FE96E020E85
:10603000EA22EF50E66EC9DEE552DF50DF2AEA6A57
:10604000000FE96E020EEA22010EEFCFDBFF010E18
:10605000DBCFE6FFBADEE552DF50DF2AEA6A000F47
:10606000E96E020EEA22EF50E66EAFDEE552010E57
:10607000DB06010EDB500008EFE3C1D0DF50DF2A62
:10608000EA6A000FE96E020EEA22EF50E66E9DDE2C
:10609000E552DF50DF2AEA6A000FE96E020EEA22BB
:1060A000010EEFCFDBFF010EDBCFE6FF8EDEE55208
:1060B000DF50DF2AEA6A000FE96E020EEA22EF5093
:1060C000E66E83DEE552010EDB06010EDB500008B2
:1060D000EFE395D0DF50DF2AEA6A000FE96E020E87
:1060E000EA22EF50E66E71DEE552DF50DF2AEA6AFF
:1060F000000FE96E020EEA22010EEFCFDBFF010E68
:10610000DBCFE6FF62DEE552DF50DF2AEA6A000FEE
:10611000E96E020EEA22EF50E66E57DEE552010EFE
:10612000DB06010EDB500008EFE369D0DF50DF2A09
:10613000EA6A000FE96E020EEA22EF50E66E45DED3
:10614000E5525DD0DF2A5BD0DF50DF2AEA6A000F1C
:10615000E96E020EEA22EF50E66E37DEE552DF50BE
:10616000DF2AEA6A000FE96E020EEA22EF50E66EBD
:106170002CDEE552DF50DF2AEA6A000FE96E020EDC
:10618000EA22EF50E66E21DEE55239D0DF50DF2AF9
:10619000EA6A000FE96E020EEA22EF50E66E15DEA3
:1061A000E552DF50DF2AEA6A000FE96E020EEA22AA
:1061B000EF50E66E0ADEE552DF50DF2AEA6A000F92
:1061C000E96E020EEA22EF50E66EFFDDE552DF5087
:1061D000DF2AEA6A000FE96E020EEA22EF50E66E4D
:1061E000F4DDE552DF50DF2AEA6A000FE96E020EA5
:1061F000EA22EF50E66EE9DDE55201D0DF2A400EDB
:10620000DF5C01E26BD6020EE15C02E2E16AE5527C
:10621000E16EE552E7CFD9FF1200D9CFE6FFE1CF1B
:10622000D9FF020EE126ECDC0401400EB06FE5DD83
:10623000DF6EDF50AB0A01E1D1D0070A01E1CCD01B
:10624000060A01E1C9D0030A01E1C3D0010A01E154
:10625000BDD00F0A01E1B7D0010A01E19CD0030AC9
:1062600001E18AD0010A01E185D0050A6BE0010A4B
:1062700053E0FA0A50E0DC0A4CE0030A48E0010A65
:1062800036E0070A2BE0040A25E0050A21E0030AAC
:1062900011E0010A01E0A5D0B0DDE76E010EE7CF05
:1062A000DBFFABDDE66E010EDBCFE6FF60D9E5522A
:1062B000E55299D0A2DDE76E010EE7CFDBFF9DDD51
:1062C000E66E010EDBCFE6FFB0D9E552E5528BD08A
:1062D000166A176A92DD186E90DD85D0161C166E50
:1062E000171C176E8ADD161A88DD171A7CD085DD1B
:1062F000586E83DD596E81DD5A6E7FDD5B6E81D80D
:10630000000904E1010E196EAD0EDF6E6CD003D9E9
:106310006AD021D968D067D070DDE76E010EE7CF73
:10632000DBFF010EDBCFE6FF68DDE66EB7EC15F0B4
:10633000E552E55262DDE66EDCEC16F0E552020154
:10634000FA6F51D05ADD0001E06F57DDE66EDCECEC
:1063500016F0E552010F0001E16F020E0001E15D50
:106360000001E26F4ADDE66EDCEC16F0E552020158
:10637000FB6F39D0B6D937D040DDE76E010EE7CFDD
:10638000DBFF3BDDE66E010EDBCFE6FF3EEC19F0F6
:10639000E552E55228D031DDE76E010EE7CFDBFF95
:1063A000010EDBCFE6FFC9EC35F0E552010EDBCF85
:1063B000E6FF000EE66E020EE66EF3EC1CF0E55210
:1063C000E552E55210D071EC17F00DD0E6EC35F047
:1063D0000AD069EC17F007D04ED805D08FEC19F031
:1063E00002D0AD0EDF6EAD0EDF5C01E020D7020EF5
:1063F000E15C02E2E16AE552E16EE552E7CFD9FFE6
:10640000120069EC17F0010EE66EE66A3EEC19F038
:10641000E552E552010EE66E020EE66E3EEC19F014
:10642000E552E552010EE66E010EE66E3EEC19F005
:10643000E552E5520001EA51EA2BEA6A600FE96E83
:10644000000EEA22EF5058160001EA51EA2BEA6AE0
:10645000600FE96E000EEA22EF50591669EC17F052
:106460005A50585C05E15B50595C02E1010E02D0C4
:10647000000E00D01200D9CFE6FFE1CFD9FF040E05
:10648000E126160EDE6E000EDD6E020EDB6A020ED7
:10649000DBCF1FF00001EB511F5C000EEC552FE22B
:1064A0000001EA51EA2BEA6A600FE96E000EEA2267
:1064B000030EEFCFDBFF185013E0020EDBA00ED06F
:1064C00018A003D0030EDB9E08D0030EDB92DB94F2
:1064D000DB96DB98DB9ADB9CDB9E02D0030EDB9025
:1064E000030EDB501F6E206ADECFE9FFDDCFEAFF2F
:1064F0001F50EE262050ED22020EDB2AC8D769EC91
:1065000017F0040EE15C02E2E16AE552E16EE55249
:10651000E7CFD9FF120069EC17F0010EE66EE66ACC
:106520003EEC19F0E552E552010EE66E0D0EE66EF8
:106530003EEC19F0E552E552010EE66E010EE66EF4
:106540003EEC19F0E552E552600E000161151A6E3D
:1065500069EC17F012001A5001010113010EE66EEA
:106560000F0EE66E3EEC19F0E552E5521200D9CF5F
:10657000E6FFE1CFD9FF71EC17F069EC17F00201EB
:10658000E351E32BEA6A000FE96E010EEA22FE0EE8
:10659000DBCFEFFF0201E351E32BEA6A000FE96E64
:1065A000010EEA22FD0EDBCFEFFF0201E351E32BE8
:1065B000EA6A000FE96E010EEA22EF6A030E020199
:1065C000E527000E0201E623010EE66EE66A3EECC8
:1065D00019F0E552E552010EE66E140EE66E3EEC41
:1065E00019F0E552E552010EE66E010EE66E3EEC44
:1065F00019F0E552E5520001EA51EA2BEA6A600F10
:10660000E96E000EEA22EF50146E0001EA51EA2B07
:10661000EA6A600FE96E000EEA22EF50156E69EC2F
:1066200017F0E552E7CFD9FF1200D9CFE6FFE1CF4F
:10663000D9FF71EC17F069EC17F00201E351E32B7D
:10664000EA6A000FE96E010EEA22FE0EDBCFEFFFD1
:106650000201E351E32BEA6A000FE96E010EEA2220
:10666000FD0EDBCFEFFF0201E351E32BEA6A000FDF
:10667000E96E010EEA22EF6A0201E351E32BEA6AB6
:10668000000FE96E010EEA2214C0EFFF0201E35190
:10669000E32BEA6A000FE96E010EEA2215C0EFFF54
:1066A000050E0201E527000E0201E623010EE66E4B
:1066B000E66A3EEC19F0E552E552010EE66E150E63
:1066C000E66E3EEC19F0E552E552010EE66E010E63
:1066D000E66E3EEC19F0E552E552E552E7CFD9FF00
:1066E0001200D9CFE6FFE1CFD9FF0A0EE126FDEC7B
:1066F0002EF0E66ED950060FE96EDACFEAFFE552CA
:10670000E750EE6EED6AFDEC2EF0E66ED950040F08
:10671000E96EDACFEAFFE552E750EE6EED6A040E5D
:10672000DBCF08F0050EDBCF09F0080E08C0DBFF59
:10673000090E09C0DBFF040EDBCF1FF0050EDBCF17
:1067400020F0203404E21F503D08000E205403E2E4
:106750000001E88D14D2020EDB6A030EDB6ADE6AEA
:10676000DD6ADECF1FF0DDCF20F0D890205004E6A8
:10677000200E1F5C000E205823E2DECFE9FFDDCFA4
:10678000EAFF030EEA02F3CFEAFF030EE902F3CFBA
:10679000E9FFF450EA26800EE926020EEA22EF50C5
:1067A0001F6E206AD950020FE96EDACFEAFF1F5040
:1067B000EE262050ED22DF2A010E01E3DB2AD1D79D
:1067C000060EDBCFE9FF070EDBCFEAFF030EEA027E
:1067D000F3CFEAFF030EE902F3CFE9FFF450EA2614
:1067E000800EE926020EEA22EF501F6E206AD95071
:1067F000020FE96EDACFEAFF1F50EE5E2050ED5A2D
:10680000040EDBCF1FF0050EDBCF20F0020EDBCF36
:1068100021F0030EDBCF22F0000ED8802156030EAC
:10682000225622502018E8AE02D0203404D01F5047
:10683000215C2050225803E20001E88DA0D1060E11
:10684000DBCF1FF0070EDBCF20F0203404E21F5017
:106850001F08000E205403E20001E88D90D1060EBF
:10686000DBCFE9FF070EDBCFEAFF030EEA02F3CF2F
:10687000EAFF030EE902F3CFE9FFF450EA26800EA7
:10688000E926020EEA22EF5001E106D1060EDBCF27
:10689000E9FF070EDBCFEAFF030EEA02F3CFEAFFC0
:1068A000030EE902F3CFE9FFF450EA26800EE92651
:1068B000020EEA22EF501F6E206A000ED8801F568B
:1068C000030E20561F06000E205A040E1FC0DBFFC9
:1068D000050E20C0DBFF060EDBCFE9FF070EDBCF86
:1068E000EAFF030EEA02F3CFEAFF030EE902F3CF59
:1068F000E9FFF450EA26800EE926020EEA22EE5263
:10690000EECFDEFFEDCFDDFFDECF1FF0DDCF20F0DD
:10691000040EDBCF21F0050EDBCF22F02050221831
:10692000E8AE02D0223404D021501F5C22502058FF
:1069300035E2060EDBCFE9FF070EDBCFEAFF030EE1
:10694000EA02F3CFEAFF030EE902F3CFE9FFF450C6
:10695000EA26800EE926020EEA22EF500001206AA4
:10696000F4251F6EF5512022DE501F24E96EDD5004
:106970002020EA6EEF50E66EDE500001F4250F0194
:10698000E96EDD500001F5210F01EA6EE552E75096
:10699000EF6EDF2A010E01E3DB2AB6D7DE6ADD6A7D
:1069A000DECF1FF0DDCF20F0D890205004E6200E7F
:1069B0001F5C000E205870E2DECFE9FFDDCFEAFF5A
:1069C000030EEA02F3CFEAFF030EE902F3CFE9FF79
:1069D000F450EA26800EE926020EEA22EECF1FF0DE
:1069E000EECF20F0EFCF21F0060EDBCFE9FF070E50
:1069F000DBCFEAFF030EEA02F3CFEAFF030EE90260
:106A0000F3CFE9FFF450EA26800EE926020EEA22CF
:106A1000EE52EECF22F0EFCF23F0000123502118E9
:106A2000E8AE02D0213404D02050225C21502358FB
:106A30002EE2060EDBCFE9FF070EDBCFEAFF030EE7
:106A4000EA02F3CFEAFF030EE902F3CFE9FFF450C5
:106A5000EA26800EE926020EEA22EF501F6E206A17
:106A6000DECFE9FFDDCFEAFF030EEA02F3CFEAFF54
:106A7000030EE902F3CFE9FFF450EA26800EE9267F
:106A8000020EEA22EE521F50EE5E2050ED5ADF2A2F
:106A9000010E01E3DB2A84D7060EDBCFE9FF070EE8
:106AA000DBCFEAFF030EEA02F3CFEAFF030EE902AF
:106AB000F3CFE9FFF450EA26800EE926020EEA221F
:106AC000080EDBCFEFFF060EDBCFE9FF070EDBCFB3
:106AD000EAFF030EEA02F3CFEAFF030EE902F3CF67
:106AE000E9FFF450EA26800EE926020EEA22EE5271
:106AF000020EDBCFEEFF030EDBCFEDFFDE6ADD6AB9
:106B0000DECF1FF0DDCF20F0060EDBCFE9FF070E52
:106B1000DBCFEAFF030EEA02F3CFEAFF030EE9023E
:106B2000F3CFE9FFF450EA26800EE926020EEA22AE
:106B3000EF50000120AE02D0D89003D01F5C000EB1
:106B400020581DE2FDEC2EF0E66E020EDB50000137
:106B5000F42500011F6E030EDB500001F52100013A
:106B6000206EDE501F24E96EDD502020EA6EE552D3
:106B7000E750EF6EDF2A010E01E3DB2AC1D70A0ED0
:106B8000E15C02E2E16AE552E16EE552E7CFD9FF4E
:106B90001200D9CFE6FFE1CFD9FFE652DF6AFE0E41
:106BA000DB50DF5C0EE2FDEC2EF0E66EDF50EA6AB1
:106BB000000FE96E020EEA22E552E750EF6EDF2A7F
:106BC000EED7E552E552E7CFD9FF1200D9CFE6FF65
:106BD000E1CFD9FF040EE126FDEC2EF0E66ED95090
:106BE000020FE96EDACFEAFFE552E750EE6EED6A8A
:106BF000020EDB500201E52500011F6E030EDB5083
:106C00000201E6210001206E000ED8801F54010E03
:106C1000205403E20001E88F36D0DE6ADD6ADECF61
:106C20001FF0DDCF20F0020EDBCF21F0030EDBCF13
:106C300022F021501F5C2250205825E2FDEC2EF05E
:106C4000E66E0201E351E32BEA6A000FE96E010EE2
:106C5000EA22E552E750EF6E0201E3511F6E206A0F
:106C6000D890205004E6000E1F5C010E205802E36D
:106C70000201E36B0201E52B000EE623DF2A010E81
:106C800001E3DB2ACCD7040EE15C02E2E16AE552C3
:106C9000E16EE552E7CFD9FF1200D9CFE6FFE1CF91
:106CA000D9FFE652DF6A81AA14D0FE0EDB50D880ED
:106CB000DF5408E3DF50DF2A010BE8B08B80E8A047
:106CC0008B9001D0DF6AF00EE66E47EC3EF0E552A5
:106CD000EAD7E552E552E7CFD9FF12006C500CE13C
:106CE0006896040100513C0BE842E8420D0802E1BD
:106CF0000ED801D04BD808D0040E6C5C03E1689626
:106D000057D802D0000E02D0010E00D01200D9CF09
:106D1000E6FFE1CFD9FFE652040104AF02D004013F
:106D2000046B0201F96B0201F16B0201F26B0201CB
:106D3000F76BF86B34EC3CF0DF6ADF501F6E206AB3
:106D4000010E1F5C000E20581BE20201F25101E00F
:106D500017D0F76ADF34FE0BF736F66E660EF626AE
:106D6000780EF7220900F5CF1FF00800F5CF20F0CC
:106D700004D020C0FAFF1F50F96EFBDFDF2ADDD7F9
:106D800005D9E552E552E7CFD9FF1200020E020104
:106D9000F15D0CE1B9D8040100BD04D00401C80EB6
:106DA000006F03D00401880E006F01D03ED912009D
:106DB000040E0001ED5D0CE112C46EFF6E50000880
:106DC00004E20001050EED6F03D00001030EED6F2C
:106DD0000201F10514E115D8020E0201F95D04E18A
:106DE0000401840E046F0AD0040104BD04D0040120
:106DF000C80E046F03D00401880E046F01D015D9AA
:106E00001200D9CFE6FFE1CFD9FF020EE126020141
:106E1000080EF75D000EF85912E2F7C2DEFFF8C265
:106E2000DDFF0201F95104E10201010EF96F06D004
:106E30000201F90503E10201020EF96F03D0080E09
:106E4000DE6EDD6A0401049304010491010EDB503F
:106E500004010413DFCF05F4000EDB500201F75FDD
:106E6000010EDB500201F85B0201180EF56F040EF3
:106E7000F66F0001EEA320D0D9CFE9FFDACFEAFF09
:106E8000EE50ED1018E0F3C2F6FFF4C2F7FF080071
:106E9000F550F5C2E9FFF6C2EAFFEF6E0201F52BED
:106EA000000EF6230201F32B000EF423DF06010E81
:106EB00001E2DB06E1D71ED0D9CFE9FFDACFEAFF46
:106EC000EE50ED1017E0F3C2E9FFF4C2EAFFEF5015
:106ED000F5C2E9FFF6C2EAFFEF6E0201F52B000EE4
:106EE000F6230201F32B000EF423DF06010E01E26C
:106EF000DB06E2D7020EE15C02E2E16AE552E16EF6
:106F0000E552E7CFD9FF1200D9CFE6FFE1CFD9FF95
:106F1000020EE126030E04010015E76E010EE7CF15
:106F2000DBFF01C4DFFFDE500201F727DD50020165
:106F3000F8230201180EF36F040EF46FD9CFE9FFA6
:106F4000DACFEAFFEE50ED1017E0F3C2E9FFF4C22A
:106F5000EAFFEF50F5C2E9FFF6C2EAFFEF6E020169
:106F6000F52B000EF6230201F32B000EF423DF06AF
:106F7000010E01E2DB06E2D7020EE15C02E2E16A09
:106F8000E552E16EE552E7CFD9FF12006D9802019C
:106F9000F2510FE10401080E016F0401100E026F9F
:106FA000040E036F0401840E006F0401840E046F4D
:106FB0003BD0040110AF25D00201F7510401165D4A
:106FC0000201F8510401175904E216C4F7F217C47C
:106FD000F8F217DF0201010EF16F0401080E016FD4
:106FE0000401100E026F040E036F0401800E006F87
:106FF0000401180E066F040E076F0401C80E046F1B
:1070000013D00201020EF16F0401056B0401C80EDA
:10701000046F0401080E016F0401180E026F040EC4
:10702000036F0401C80E006F12000201F16B04012E
:10703000080E016F0401100E026F040E036F0401AD
:107040008C0E006F0401046B12008986899454B081
:10705000898492940000899655A08994898655B0B8
:107060008984569E8996898692848996898680B479
:10707000568E899612005438556E5638576E5AC03F
:107080005CF05BC05DF0FE0E5A6E040E5B6E06EEA9
:1070900000F0EE6AEAA6FDD7120007EEFFF0BAD8BC
:1070A0005CC05AF05DC05BF08038ED125D6EEA8224
:1070B00000D000D000D00ED081AAA9D08038ED1227
:1070C000EA825D6E551457181EE15C5058140EE1AB
:1070D000594EAAD08050EF6E5C6E5414561816E1CB
:1070E0005D385814E9E1592EE9D7AAD00000805044
:1070F000EF6E5C6E5414561809E15D385814DCE1EB
:10710000592EDCD79DD081AA82D0E4D70000D4D7F5
:1071100007EEFFF07FD85CC05AF05DC05BF08038AE
:10712000ED125D6EEA8200D000D000D00ED081AAB0
:107130006ED08038ED12EA825D6E551457181EE14C
:107140005C5058140EE0594E6FD08050EF6E5C6E5C
:107150005414561816E15D385814E9E0592EE9D751
:107160006FD000008050EF6E5C6E5414561809E129
:107170005D385814DCE0592EDCD762D081AA47D0A4
:10718000E4D70000D4D707EEFFF044D85CC05AF033
:107190005DC05BF07DD800008038ED125D6EEA8244
:1071A00000D000D000D0000010D081AA30D070D81C
:1071B0008038ED12EA825D6E5514571823E15C5059
:1071C00058145F1810E1594E2FD062D88050EF6EDE
:1071D0005C6E5414561819E15D3858145F18E5E1D7
:1071E000592EE5D72DD0000053D88050EF6E5C6E3D
:1071F000541456180AE15D3858145F18D6E1592E18
:10720000D6D71ED081AA03D0E0D700D0CED7400E6B
:10721000556E12008050EF6E00D000D000D00000FC
:107220005E5227E035D825D08050EF6EE9CF54F07C
:10723000EA508009556E00D05E521BE029D819D063
:107240008038ED12EA82E9CF54F0EACF55F000D051
:107250005E5202E01DD800D08050EF6E00005A2E22
:1072600015D05B4E1200000000005E5202E010D804
:1072700000D08038ED12EA825A2E09D05B4E1200FF
:10728000000000005E52E8E003D8E6D7EDD7F9D75A
:107290005E5000D000D00000E84E120000D0000088
:1072A000F8D700EE00F00F0EEE6AEA62FDD712008A
:1072B000040110511F0B010801E07DD0040114519D
:1072C00001E079D0060E0401115D2FE10401135194
:1072D000230A28E0010A13E0030A01E024D0020196
:1072E000020EF26F0001EF0505E102013C0EF36FA3
:1072F000770EF46F090E0201F76FF86B14D00201DC
:10730000020EF26F0001EF0505E102013B0EF36F83
:10731000780EF46F0001EF0504E11D0E0201F76F16
:10732000F86B01D000D00001EE8304011051600B16
:10733000E842E842E842E842E842010801E03BD086
:10734000040111510B0A31E0080A21E0090A19E091
:10735000080A09E00B0A05E0080A01E02CD02CD845
:107360002AD02BD828D00201020EF26F0201F10EB2
:10737000F36F000EF46F0001EE930201010EF76F40
:107380001AD00201020EF26F13C4F1F014D0020100
:10739000020EF26F0201F20EF36F000EF46F0001A5
:1073A000EE930201010EF76F06D00201020EF26F9A
:1073B00012C4F2F000D01200120012000001F36BB0
:1073C0001E0E716E0401400E096F0401200E0A6F3B
:1073D000040E0B6F0401880E086F0401600E0E6F1F
:1073E000040E0F6F0401400E0C6F1200D9CFE6FFA0
:1073F000E1CFD9FFE652FC0EDB50400805E2400E1B
:10740000F36EFC0EF3CFDBFFDF6AFC0EDB50DF5CBC
:1074100019E2DF50E76EFD0EDBCFE9FFFE0EDBCF9A
:10742000EAFFE750E926000EEA22EF50E66EDF5051
:10743000EA6A600FE96E040EEA22E552E750EF6E49
:10744000DF2AE3D7FC0EDBCF0DF4400E04010C174E
:1074500004010C7D880E04010C13E552E552E7CFC0
:10746000D9FF1200D9CFE6FFE1CFD9FF0001F36BBE
:10747000040108BF39D0FC0EDBCF1FF00401095115
:10748000D8801F5403E2FC0E09C4DBFF0001F36B3C
:10749000FC0EDB500001F35D1CE20001F351EA6ACF
:1074A000200FE96E040EEA22EF50E66E0001F35160
:1074B000E76EFD0EDBCFE9FFFE0EDBCFEAFFE75004
:1074C000E926000EEA22E552E750EF6E0001F32BA9
:1074D000DFD70401400E096F400E040108170401B4
:1074E000087D880E040108130001F35100D0E55215
:1074F000E7CFD9FF1200D8CFE4FFE0CFE4FFE46E7E
:10750000DACFE4FFE2CFDAFFE6520001E8A37CD055
:10751000A150400B1DE0A050400B1AE0B4BE17D0A4
:10752000A09CCD981550CF6E480E1424296E2A6A5F
:10753000000E2A222A3404E22950FF08000E2A54A1
:1075400001E2CF2A480E1424CE6E9E909D80A19C0D
:107550009E50010B31E09D50010B2EE01550CF6E77
:107560001450CE6E9E9016500AE1CD88B4AE04D071
:107570009D90A19CA08C02D08B80162A1DD0165005
:10758000080815E2B4AE0DD01DA003D017501B6E35
:1075900007D01DA203D017501C6E02D017501A6ED0
:1075A0001D2A8B90166A9D90A19CA08C05D01790E7
:1075B0001742B4BE178E162AA150020B24E0A05029
:1075C000020B21E01550B36E1450B26EA192185008
:1075D00004E18996182A8B8016D0090E185C03E105
:1075E0008986182A10D01850090804E2186AA09257
:1075F0008B9009D0010E1914E8B08986E8A089960D
:10760000182A1990194262D09EA035D09E90FA0E89
:10761000CF6E380ECE6E8150100B10E10201FA5180
:10762000C45C0CE20C0E0201FC5D05E18A948A88C0
:107630000001E78902D00201FC2B02D00201FC6BA1
:10764000300E0001E71512E00201FEC229F0FFC270
:107650002AF0FE2B000EFF239B0ED8802954020E29
:107660002A5404E28B700201FE6BFF6B9E9C010E9C
:10767000C26E9D8CC2829EAC29D09E9C0C0EBA5CC0
:1076800021E10001E151D880C45401E2BB6A00014C
:10769000E251C45C02E2E0C0BBFF8150040B10E089
:1076A0000201FB51C45C0CE20C0E0201FD5D05E120
:1076B0008A948A880001E78B02D00201FD2B02D058
:1076C0000201FD6B050EC26E9D9CC282A1B4FF003B
:1076D000E552E5CFDAFFE550E5CFE0FFE5CFD8FF93
:1076E00010000201FC6B0201FD6B800ECD6EFA0EE4
:1076F000CF6E380ECE6E9E909D80CD809E9C9D9CC0
:10770000260EC06E050EC26EC28212009D90CD90F4
:10771000C26A9E9C9D9C120012010002000000089B
:10772000D80433000200010200020902290001010D
:107730000280320904000002030000000921010058
:107740000001221D00070581034000010705010318
:1077500040000109022000010204803209040000F7
:1077600002FF000000070581034000010705010337
:107770004000010403090434034D006900630072F2
:10778000006F00630068006900700020005400650D
:1077900000630068006E006F006C006F0067007986
:1077A00000200049006E0063002E0048035000498D
:1077B0000043006B00690074002000320020004D7F
:1077C000006900630072006F0063006F006E007458
:1077D0000072006F006C006C0065007200200050A9
:1077E0000072006F006700720061006D006D00653F
:1077F0000072001603500049004300310038004673
:10780000003200350035003000320350004900439B
:10781000006B006900740020003200200043006FFC
:10782000006E0066006900670075007200610074F8
:107830000069006F006E00200032000600FF0901A1
:10784000A10119012940150026FF00750895408106
:1078500002190129409102C02A775377737777770D
:10786000AB77F3770978B07204011051600BE842EE
:10787000E842E842E842E842000901E08BD0040116
:107880001151080A01E177D0010A63E00F0A0AE00A
:10789000030A01E07ED00201010EF26F0001040E26
:1078A000ED6F78D00201010EF26F040113050AE1B9
:1078B0000201180EF36F770EF46F120E0201F76FCC
:1078C000F86B44D0020E0401135D1FE10401125154
:1078D000F66EF76AD890F636F736580EF626780E1A
:1078E000F7220900F5CFF3F20A00F5CFF4F2020E09
:1078F0000201F76AF325F66EF451F7220900F5CF7D
:10790000F7F20A00F5CFF8F221D0030E0401135D5F
:107910001BE104011251F66EF76AD890F636F7367D
:107920005C0EF626780EF7220900F5CFF3F20A0076
:10793000F5CFF4F2F3C2F6FFF4C2F7FF0800F550FA
:107940000201F76FF86B02D00201F26B0001EE83C7
:1079500021D00201010EF26F12C4EFF004011251A6
:1079600004E10001050EED6F05D00001060EED6F7C
:10797000DEEC39F00FD00201010EF26F0201EF0EC2
:10798000F36F000EF46F0001EE930201010EF76F2A
:1079900001D000D0120009C013F008C012F0085046
:1079A0000D02F4CF07F0F3CF06F009500E02F4CF2A
:1079B00009F0F3CF08F00D02F3500726F450082227
:1079C000E86A092212500E02F3500726F4500822EA
:1079D000E86A09220EAEF1EF3CF01250085E135037
:1079E000095A13AE000C0D50085E0E50095A000CD7
:1079F00008C012F008500D02F4CF07F0F3CF06F0E4
:107A000009500E02F4CF09F0F3CF08F00D02F35045
:107A10000726F4500822E86A092212500E02F35099
:107A20000726F4500822E86A0922000C09C013F066
:107A300008C012F007C011F007500C02F4CF05F097
:107A4000F3CF04F008500D02F4CF07F0F3CF06F0A7
:107A50000C02F3500526F4500622E86A0722115062
:107A60000D02F3500526F4500622E86A0722095059
:107A70000C02F3500626F450072209500D02086A42
:107A8000E86A0822F3500726F450082211500E022B
:107A9000F3500626F4500722096AE86A08220922F0
:107AA00012500E02F3500726F4500822E86A092209
:107AB00013500E02F3500826F4500922000C080E51
:107AC0006D6E6DBAFED7686A110E696E0001020E06
:107AD000ED6F12006D6A696A0001ED6B120068506B
:107AE000040B09E06950040B06E06D92699468A4E8
:107AF00002D06894FCD76850010B04E06950010B78
:107B000001E025D86850200B06E06950200B03E007
:107B100070B07090689A030E0001ED5D01E216D01E
:107B20000001F66B040E0001F65D10E26850080BD0
:107B300009E06950080B06E06EEC36F0000901E13F
:107B4000689601D003D00001F62BECD71200686ACA
:107B50007B0E696E6E6A160E706E68A608D0689607
:107B6000000000000000000000000000F6D76D9843
:107B700015EC38F00001EF6B0001030EED6F120001
:107B8000F20EF66E5B0EF76E000EF86E0201090043
:107B9000F550EC6F0900F550ED6F03E1EC6701D093
:107BA0003DD00900F550E76F0900F550E86F090076
:107BB000F550E96F09000900F550E96E0900F5502C
:107BC000EA6E090009000900F550EA6F0900F55056
:107BD000EB6F09000900F6CFEEF2F7CFEFF2F8CF26
:107BE000F0F2E7C2F6FFE8C2F7FFE9C2F8FF0201D0
:107BF000EA5302E1EB5307E00900F550EE6EEA07A5
:107C0000F8E2EB07F9D7EEC2F6FFEFC2F7FFF0C2DA
:107C1000F8FF0201EC07000EED5BBFD71200065023
:107C20000B02F3CF02F0F4CF03F00C02F350032663
:107C3000000EF420046E06500D02F3500426000ED0
:107C4000F420056E06500E02F350052607500B0275
:107C5000F3500326F4500422000E052207500C02B4
:107C6000F3500426F450052207500D02F350052668
:107C700008500B02F3500426F450052208500C0261
:107C8000F350052609500B02F35005261200FF0E93
:107C9000E3502C6EEF0E01D0F30EE76EE72E4EEFA1
:107CA0003EF00C0E2B6EE76AE72E54EF3EF02B2EC3
:107CB00053EF3EF02C2E4CEF3EF0120006D86FEC46
:107CC0003DF0D5EC10F0FBD71200140E6F6E0001E2
:107CD000ED6B0001EE6B0001EF6B15EC10F05FEC4B
:107CE0003DF0120013EE00F023EE00F0F86A019C64
:107CF000C0EC3DF099EC3EF05EEC3EF0FBD712009C
:107D0000FF0EE3502C6E1B0E00D001D0200EE76E4C
:107D1000E72EFED72C2EFAD700D01200FF0EE3502C
:107D2000E84E1200000000D000D000D0E82EFAD7B4
:107D3000120012000005FFFFFFFFFFFFFFFFFFFF24
:107D4000FFFFFFFFFFFFFFFFFFFFFFFFFFFFFFFF43
:107D5000FFFFFFFFFFFFFFFFFFFFFFFFFFFFFFFF33
:107D6000FFFFFFFFFFFFFFFFFFFFFFFFFFFFFFFF23
:107D7000FFFFFFFFFFFFFFFFFFFFFFFFFFFFFFFF13
:107FF000FFFFFFFFFFFFFFFFFFFFFFFFFFFF5555E5
:0200000400F00A
:1000000000FFFFFFFFFFFFFFFFFFFFFFFFFFFFFFFF
:10001000FFFFFFFFFFFFFFFFFFFFFFFFFFFFFFFFF0
:10002000FFFFFFFFFFFFFFFFFFFFFFFFFFFFFFFFE0
:10003000FFFFFFFFFFFFFFFFFFFFFFFFFFFFFFFFD0
:10004000FFFFFFFFFFFFFFFFFFFFFFFFFFFFFFFFC0
:10005000FFFFFFFFFFFFFFFFFFFFFFFFFFFFFFFFB0
:10006000FFFFFFFFFFFFFFFFFFFFFFFFFFFFFFFFA0
:10007000FFFFFFFFFFFFFFFFFFFFFFFFFFFFFFFF90
:10008000FFFFFFFFFFFFFFFFFFFFFFFFFFFFFFFF80
:10009000FFFFFFFFFFFFFFFFFFFFFFFFFFFFFFFF70
:1000A000FFFFFFFFFFFFFFFFFFFFFFFFFFFFFFFF60
:1000B000FFFFFFFFFFFFFFFFFFFFFFFFFFFFFFFF50
:1000C000FFFFFFFFFFFFFFFFFFFFFFFFFFFFFFFF40
:1000D000FFFFFFFFFFFFFFFFFFFFFFFFFFFFFFFF30
:1000E000FFFFFFFFFFFFFFFFFFFFFFFFFFFFFFFF20
:1000F000FFFFFFFFFFFFFFFFFFFFFFFFFFFFFFFF10
:020000040030CA
:0E000000240E391E000181000FC00EA00F401B
:020000040020DA
:08000000FFFFFFFFFFFFFFFF00
:00000001FF
